 jli

 Timestamp is ffffffff (Sun Feb  7 06:28:15 2106)

 Preferred load address is 10000000

 Start         Length     Name                   Class
 0001:00000000 00009c29H .text$mn                CODE
 0002:00000000 0000019cH .idata$5                DATA
 0002:0000019c 00000004H .00cfg                  DATA
 0002:000001a0 00000004H .CRT$XCA                DATA
 0002:000001a4 00000004H .CRT$XCZ                DATA
 0002:000001a8 00000004H .CRT$XIA                DATA
 0002:000001ac 00000004H .CRT$XIZ                DATA
 0002:000001b0 00000004H .CRT$XPA                DATA
 0002:000001b4 00000004H .CRT$XPZ                DATA
 0002:000001b8 00000004H .CRT$XTA                DATA
 0002:000001bc 00000004H .CRT$XTZ                DATA
 0002:000001c0 00000000H .gfids$y                DATA
 0002:000001c0 00005110H .rdata                  DATA
 0002:000052d0 00000004H .rdata$sxdata           DATA
 0002:000052d4 00000280H .rdata$zzzdbg           DATA
 0002:00005554 00000004H .rtc$IAA                DATA
 0002:00005558 00000004H .rtc$IZZ                DATA
 0002:0000555c 00000004H .rtc$TAA                DATA
 0002:00005560 00000008H .rtc$TZZ                DATA
 0002:00005568 00000088H .xdata$x                DATA
 0002:000055f0 00000274H .edata                  DATA
 0002:00005864 000000dcH .idata$2                DATA
 0002:00005940 00000014H .idata$3                DATA
 0002:00005954 0000019cH .idata$4                DATA
 0002:00005af0 000006caH .idata$6                DATA
 0003:00000000 00000068H .data                   DATA
 0003:00000068 0000056cH .bss                    DATA
 0004:00000000 00000060H .rsrc$01                DATA
 0004:00000060 00000300H .rsrc$02                DATA

  Address         Publics by Value              Rva+Base       Lib:Object

 0000:00000000       ___guard_iat_table         00000000     <absolute>
 0000:00000000       ___guard_longjmp_count     00000000     <absolute>
 0000:00000000       ___guard_fids_table        00000000     <absolute>
 0000:00000000       ___dynamic_value_reloc_table 00000000     <absolute>
 0000:00000000       ___hybrid_code_map         00000000     <absolute>
 0000:00000000       ___hybrid_auxiliary_iat    00000000     <absolute>
 0000:00000000       ___enclave_config          00000000     <absolute>
 0000:00000000       ___volatile_metadata       00000000     <absolute>
 0000:00000000       ___hybrid_code_map_count   00000000     <absolute>
 0000:00000000       ___guard_longjmp_table     00000000     <absolute>
 0000:00000000       ___guard_fids_count        00000000     <absolute>
 0000:00000000       ___guard_iat_count         00000000     <absolute>
 0000:00000001       ___safe_se_handler_count   00000001     <absolute>
 0000:00000100       ___guard_flags             00000100     <absolute>
 0000:00000000       ___ImageBase               10000000     <linker-defined>
 0001:00000000       _JLI_AddArgsFromEnvVar@8   10001000 f   args.obj
 0001:0000004c       _JLI_GetAppArgIndex@0      1000104c f   args.obj
 0001:00000052       _JLI_InitArgProcessing@8   10001052 f   args.obj
 0001:0000008b       _JLI_PreprocessArg@8       1000108b f   args.obj
 0001:00000405       _isTerminalOpt             10001405 f   args.obj
 0001:0000087f       _JLI_CmdToArgs@4           1000187f f   cmdtoargs.obj
 0001:000009f2       _JLI_GetStdArgc@0          100019f2 f   cmdtoargs.obj
 0001:000009f8       _JLI_GetStdArgs@0          100019f8 f   cmdtoargs.obj
 0001:00000c7b       _inflate_fast              10001c7b f   inffast.obj
 0001:00001083       _inflate                   10002083 f   inflate.obj
 0001:000026bf       _inflateEnd                100036bf f   inflate.obj
 0001:000026fb       _inflateInit2_             100036fb f   inflate.obj
 0001:000027a1       _inflateReset              100037a1 f   inflate.obj
 0001:000027ca       _inflateReset2             100037ca f   inflate.obj
 0001:00002842       _inflateResetKeep          10003842 f   inflate.obj
 0001:000029b4       _inflate_table             100039b4 f   inftrees.obj
 0001:00002fad       _AddOption                 10003fad f   java.obj
 0001:000030fa       _CheckJvmType              100040fa f   java.obj
 0001:00003376       _ContinueInNewThread       10004376 f   java.obj
 0001:0000357e       _GetLauncherHelperClass    1000457e f   java.obj
 0001:000039b6       _IsSourceFile              100049b6 f   java.obj
 0001:000039ff       _IsWhiteSpaceOption        100049ff f   java.obj
 0001:00003a1f       _JLI_Launch@56             10004a1f f   java.obj
 0001:00003d24       _JLI_ReportMessage         10004d24 f   java.obj
 0001:00003d5a       _JLI_ShowMessage           10004d5a f   java.obj
 0001:00003d90       _JavaMain                  10004d90 f   java.obj
 0001:000043b4       _NewPlatformStringArray    100053b4 f   java.obj
 0001:00004ff9       _ReadKnownVMs              10005ff9 f   java.obj
 0001:00005624       _SetJavaCommandLineProp    10006624 f   java.obj
 0001:000058be       _ShowSplashScreen          100068be f   java.obj
 0001:00005b52       ___local_stdio_printf_options 10006b52 f i java.obj
 0001:00005b58       ___local_stdio_scanf_options 10006b58 f i java.obj
 0001:00005b5e       __vfprintf_l               10006b5e f i java.obj
 0001:00005b82       __vsnprintf_l              10006b82 f i java.obj
 0001:00005bb5       __vsscanf_l                10006bb5 f i java.obj
 0001:00005c89       _fprintf                   10006c89 f i java.obj
 0001:00005d79       _printf                    10006d79 f i java.obj
 0001:00005d97       _sprintf                   10006d97 f i java.obj
 0001:00005db1       _sscanf                    10006db1 f i java.obj
 0001:00005dc9       _AWTPreload                10006dc9 f   java_md.obj
 0001:00005f18       _CallJavaMainInNewThread   10006f18 f   java_md.obj
 0001:00006058       _Counter2Micros            10007058 f   java_md.obj
 0001:00006097       _CounterGet                10007097 f   java_md.obj
 0001:000060df       _CreateApplicationArgs     100070df f   java_md.obj
 0001:00006391       _CreateExecutionEnvironment 10007391 f   java_md.obj
 0001:000064fc       _FindBootStrapClass        100074fc f   java_md.obj
 0001:0000654a       _GetApplicationHome        1000754a f   java_md.obj
 0001:00006565       _GetApplicationHomeFromDll 10007565 f   java_md.obj
 0001:000065a0       _GetBoolParamValue         100075a0 f   java_md.obj
 0001:0000679b       _GetParamValue             1000779b f   java_md.obj
 0001:000067d1       _InitLauncher              100077d1 f   java_md.obj
 0001:00006806       _IsJavaw                   10007806 f   java_md.obj
 0001:0000680c       _JLI_Open                  1000780c f   java_md.obj
 0001:00006944       _JLI_ReportErrorMessage    10007944 f   java_md.obj
 0001:000069d0       _JLI_ReportErrorMessageSys 100079d0 f   java_md.obj
 0001:00006b01       _JLI_ReportExceptionDescription@4 10007b01 f   java_md.obj
 0001:00006b2d       _JLI_Snprintf              10007b2d f   java_md.obj
 0001:00006b73       _JVMInit                   10007b73 f   java_md.obj
 0001:00006b9d       _LoadJavaVM                10007b9d f   java_md.obj
 0001:00006d86       _PostJVMInit               10007d86 f   java_md.obj
 0001:00006d86       @_guard_check_icall_nop@4  10007d86 f   MSVCRT:guard_support.obj
 0001:00006d86       _SetJavaLauncherPlatformProps 10007d86 f   java_md.obj
 0001:00006d86       _RegisterThread            10007d86 f   java_md.obj
 0001:00006d87       _ProcessPlatformOption     10007d87 f   java_md.obj
 0001:00006d8a       _SplashProcAddress         10007d8a f   java_md.obj
 0001:00006e37       _TruncatePath              10007e37 f   java_md.obj
 0001:00006e63       _UnsetEnv                  10007e63 f   java_md.obj
 0001:00006ea8       __vscprintf_l              10007ea8 f i java_md.obj
 0001:00006ed8       __vsnprintf                10007ed8 f i java_md.obj
 0001:00006ef3       _vsnprintf                 10007ef3 f i java_md.obj
 0001:00006f25       _JLI_HasSuffix             10007f25 f   jli_util.obj
 0001:00006f52       _JLI_IsTraceLauncher       10007f52 f   jli_util.obj
 0001:00006f58       _JLI_List_add@8            10007f58 f   jli_util.obj
 0001:00006f7d       _JLI_List_addSubstring     10007f7d f   jli_util.obj
 0001:00006fbd       _JLI_List_combine          10007fbd f   jli_util.obj
 0001:00007024       _JLI_List_ensureCapacity   10008024 f   jli_util.obj
 0001:0000704e       _JLI_List_free             1000804e f   jli_util.obj
 0001:00007088       _JLI_List_join             10008088 f   jli_util.obj
 0001:000070fc       _JLI_List_new@4            100080fc f   jli_util.obj
 0001:00007122       _JLI_List_split            10008122 f   jli_util.obj
 0001:000071aa       _JLI_MemAlloc@4            100081aa f   jli_util.obj
 0001:000071d0       _JLI_MemFree@4             100081d0 f   jli_util.obj
 0001:000071de       _JLI_MemRealloc            100081de f   jli_util.obj
 0001:00007207       _JLI_SetTraceLauncher@0    10008207 f   jli_util.obj
 0001:0000722f       _JLI_StrCCmp               1000822f f   jli_util.obj
 0001:0000724b       _JLI_StringDup@4           1000824b f   jli_util.obj
 0001:00007271       _JLI_TraceLauncher         10008271 f   jli_util.obj
 0001:0000729b       _vprintf                   1000829b f i jli_util.obj
 0001:000072b8       _JLI_FreeManifest          100082b8 f   parse_manifest.obj
 0001:000072ca       _JLI_JarUnpackFile         100082ca f   parse_manifest.obj
 0001:00007322       _JLI_ManifestIterate@12    10008322 f   parse_manifest.obj
 0001:000073de       _JLI_ParseManifest         100083de f   parse_manifest.obj
 0001:000083eb       _DoSplashGetScaledImageName 100093eb f   splashscreen_stubs.obj
 0001:00008412       _DoSplashGetScaledImgNameMaxPstfixLen 10009412 f   splashscreen_stubs.obj
 0001:00008432       _DoSplashInit              10009432 f   splashscreen_stubs.obj
 0001:00008452       _DoSplashLoadFile          10009452 f   splashscreen_stubs.obj
 0001:00008472       _DoSplashLoadMemory        10009472 f   splashscreen_stubs.obj
 0001:00008492       _DoSplashSetFileJarName    10009492 f   splashscreen_stubs.obj
 0001:000084b2       _DoSplashSetScaleFactor    100094b2 f   splashscreen_stubs.obj
 0001:000085f9       _JLI_WildcardExpandClasspath 100095f9 f   wildcard.obj
 0001:000087a1       _adler32                   100097a1 f   zadler32.obj
 0001:000087a6       _adler32_z                 100097a6 f   zadler32.obj
 0001:000089e3       _crc32                     100099e3 f   zcrc32.obj
 0001:000089e8       _crc32_z                   100099e8 f   zcrc32.obj
 0001:00008cd1       _zcalloc                   10009cd1 f   zutil.obj
 0001:00008ce3       _zcfree                    10009ce3 f   zutil.obj
 0001:00008cef       @__security_check_cookie@4 10009cef f   MSVCRT:secchk.obj
 0001:00008d00       __chkstk                   10009d00 f   MSVCRT:chkstk.obj
 0001:00008d00       __alloca_probe             10009d00 f   MSVCRT:chkstk.obj
 0001:00008d2d       ___raise_securityfailure   10009d2d f   MSVCRT:gs_report.obj
 0001:00008d55       ___report_gsfailure        10009d55 f   MSVCRT:gs_report.obj
 0001:00008e4e       ___report_rangecheckfailure 10009e4e f   MSVCRT:gs_report.obj
 0001:00008e5a       ___report_securityfailure  10009e5a f   MSVCRT:gs_report.obj
 0001:00008f30       __alldiv                   10009f30 f   MSVCRT:lldiv.obj
 0001:00008fe0       __allmul                   10009fe0 f   MSVCRT:llmul.obj
 0001:00009020       __allrem                   1000a020 f   MSVCRT:llrem.obj
 0001:000093f2       __DllMainCRTStartup@12     1000a3f2 f   MSVCRT:dll_dllmain.obj
 0001:00009462       ___security_init_cookie    1000a462 f   MSVCRT:gs_support.obj
 0001:000094ad       _DllMain@12                1000a4ad f   MSVCRT:dll_dllmain_stub.obj
 0001:000094cf       ?__scrt_initialize_type_info@@YAXXZ 1000a4cf f   MSVCRT:tncleanup.obj
 0001:000094db       ?__scrt_uninitialize_type_info@@YAXXZ 1000a4db f   MSVCRT:tncleanup.obj
 0001:000094e7       ___scrt_initialize_default_local_stdio_options 1000a4e7 f   MSVCRT:default_local_stdio_options.obj
 0001:00009548       ___scrt_acquire_startup_lock 1000a548 f   MSVCRT:utility.obj
 0001:0000957a       ___scrt_dllmain_after_initialize_c 1000a57a f   MSVCRT:utility.obj
 0001:000095a5       ___scrt_dllmain_before_initialize_c 1000a5a5 f   MSVCRT:utility.obj
 0001:000095b3       ___scrt_dllmain_crt_thread_attach 1000a5b3 f   MSVCRT:utility.obj
 0001:000095d2       ___scrt_dllmain_crt_thread_detach 1000a5d2 f   MSVCRT:utility.obj
 0001:000095df       ___scrt_dllmain_exception_filter 1000a5df f   MSVCRT:utility.obj
 0001:00009613       ___scrt_dllmain_uninitialize_c 1000a613 f   MSVCRT:utility.obj
 0001:00009636       ___scrt_dllmain_uninitialize_critical 1000a636 f   MSVCRT:utility.obj
 0001:00009643       ___scrt_initialize_crt     1000a643 f   MSVCRT:utility.obj
 0001:0000967c       ___scrt_initialize_onexit_tables 1000a67c f   MSVCRT:utility.obj
 0001:00009721       ___scrt_is_nonwritable_in_current_image 1000a721 f   MSVCRT:utility.obj
 0001:000097b5       ___scrt_release_startup_lock 1000a7b5 f   MSVCRT:utility.obj
 0001:000097d2       ___scrt_uninitialize_crt   1000a7d2 f   MSVCRT:utility.obj
 0001:000097fa       ___scrt_get_dyn_tls_init_callback 1000a7fa f   MSVCRT:dyn_tls_init.obj
 0001:00009800       ___scrt_fastfail           1000a800 f   MSVCRT:utility_desktop.obj
 0001:0000991a       __crt_debugger_hook        1000a91a f   MSVCRT:utility_desktop.obj
 0001:00009922       __RTC_Initialize           1000a922 f   MSVCRT:initsect.obj
 0001:0000994e       __RTC_Terminate            1000a94e f   MSVCRT:initsect.obj
 0001:00009980       __SEH_prolog4              1000a980 f   MSVCRT:sehprolg4.obj
 0001:000099c6       __SEH_epilog4              1000a9c6 f   MSVCRT:sehprolg4.obj
 0001:000099db       __except_handler4          1000a9db f   MSVCRT:chandler4gs.obj
 0001:000099fe       ___isa_available_init      1000a9fe f   MSVCRT:cpu_disp.obj
 0001:00009b95       __get_startup_argv_mode    1000ab95 f   MSVCRT:argv_mode.obj
 0001:00009b99       ___scrt_is_ucrt_dll_in_use 1000ab99 f   MSVCRT:ucrt_detection.obj
 0001:00009ba5       _IsProcessorFeaturePresent@4 1000aba5 f   kernel32:KERNEL32.dll
 0001:00009bab       _memcpy                    1000abab f   vcruntime:VCRUNTIME140.dll
 0001:00009bb1       _strchr                    1000abb1 f   vcruntime:VCRUNTIME140.dll
 0001:00009bb7       _memset                    1000abb7 f   vcruntime:VCRUNTIME140.dll
 0001:00009bbd       _strrchr                   1000abbd f   vcruntime:VCRUNTIME140.dll
 0001:00009bc3       _memcmp                    1000abc3 f   vcruntime:VCRUNTIME140.dll
 0001:00009bc9       _memmove                   1000abc9 f   vcruntime:VCRUNTIME140.dll
 0001:00009bcf       ___std_type_info_destroy_list 1000abcf f   vcruntime:VCRUNTIME140.dll
 0001:00009bd5       __except_handler4_common   1000abd5 f   vcruntime:VCRUNTIME140.dll
 0001:00009bdb       _strcmp                    1000abdb f   ucrt:api-ms-win-crt-string-l1-1-0.dll
 0001:00009be1       _strlen                    1000abe1 f   ucrt:api-ms-win-crt-string-l1-1-0.dll
 0001:00009be7       _strcat                    1000abe7 f   ucrt:api-ms-win-crt-string-l1-1-0.dll
 0001:00009bed       _strcpy                    1000abed f   ucrt:api-ms-win-crt-string-l1-1-0.dll
 0001:00009bf3       __initterm                 1000abf3 f   ucrt:api-ms-win-crt-runtime-l1-1-0.dll
 0001:00009bf9       __initterm_e               1000abf9 f   ucrt:api-ms-win-crt-runtime-l1-1-0.dll
 0001:00009bff       __seh_filter_dll           1000abff f   ucrt:api-ms-win-crt-runtime-l1-1-0.dll
 0001:00009c05       __configure_narrow_argv    1000ac05 f   ucrt:api-ms-win-crt-runtime-l1-1-0.dll
 0001:00009c0b       __initialize_narrow_environment 1000ac0b f   ucrt:api-ms-win-crt-runtime-l1-1-0.dll
 0001:00009c11       __initialize_onexit_table  1000ac11 f   ucrt:api-ms-win-crt-runtime-l1-1-0.dll
 0001:00009c17       __execute_onexit_table     1000ac17 f   ucrt:api-ms-win-crt-runtime-l1-1-0.dll
 0001:00009c1d       __cexit                    1000ac1d f   ucrt:api-ms-win-crt-runtime-l1-1-0.dll
 0001:00009c23       ___scrt_stub_for_acrt_initialize 1000ac23 f   MSVCRT:ucrt_stubs.obj
 0001:00009c23       ___scrt_stub_for_acrt_thread_attach 1000ac23 f   MSVCRT:ucrt_stubs.obj
 0001:00009c23       ___acrt_uninitialize       1000ac23 f   MSVCRT:ucrt_stubs.obj
 0001:00009c23       ___acrt_uninitialize_critical 1000ac23 f   MSVCRT:ucrt_stubs.obj
 0001:00009c23       ___vcrt_thread_attach      1000ac23 f   MSVCRT:ucrt_stubs.obj
 0001:00009c23       ___vcrt_uninitialize       1000ac23 f   MSVCRT:ucrt_stubs.obj
 0001:00009c23       ___scrt_stub_for_acrt_uninitialize 1000ac23 f   MSVCRT:ucrt_stubs.obj
 0001:00009c23       ___vcrt_uninitialize_critical 1000ac23 f   MSVCRT:ucrt_stubs.obj
 0001:00009c23       ___acrt_initialize         1000ac23 f   MSVCRT:ucrt_stubs.obj
 0001:00009c23       ___vcrt_thread_detach      1000ac23 f   MSVCRT:ucrt_stubs.obj
 0001:00009c23       ___acrt_thread_attach      1000ac23 f   MSVCRT:ucrt_stubs.obj
 0001:00009c23       ___scrt_stub_for_acrt_uninitialize_critical 1000ac23 f   MSVCRT:ucrt_stubs.obj
 0001:00009c23       ___scrt_stub_for_acrt_thread_detach 1000ac23 f   MSVCRT:ucrt_stubs.obj
 0001:00009c23       ___vcrt_initialize         1000ac23 f   MSVCRT:ucrt_stubs.obj
 0001:00009c23       ___acrt_thread_detach      1000ac23 f   MSVCRT:ucrt_stubs.obj
 0001:00009c26       ___scrt_stub_for_is_c_termination_complete 1000ac26 f   MSVCRT:ucrt_stubs.obj
 0001:00009c26       __is_c_termination_complete 1000ac26 f   MSVCRT:ucrt_stubs.obj
 0002:00000000       __imp__InitCommonControlsEx@4 1000b000     comctl32:COMCTL32.dll
 0002:00000004       \177COMCTL32_NULL_THUNK_DATA 1000b004     comctl32:COMCTL32.dll
 0002:00000008       __imp__IsDebuggerPresent@0 1000b008     kernel32:KERNEL32.dll
 0002:0000000c       __imp__CreateFileW@28      1000b00c     kernel32:KERNEL32.dll
 0002:00000010       __imp__CloseHandle@4       1000b010     kernel32:KERNEL32.dll
 0002:00000014       __imp__GetLastError@0      1000b014     kernel32:KERNEL32.dll
 0002:00000018       __imp__QueryPerformanceCounter@4 1000b018     kernel32:KERNEL32.dll
 0002:0000001c       __imp__QueryPerformanceFrequency@4 1000b01c     kernel32:KERNEL32.dll
 0002:00000020       __imp__WaitForSingleObject@8 1000b020     kernel32:KERNEL32.dll
 0002:00000024       __imp__GetExitCodeThread@8 1000b024     kernel32:KERNEL32.dll
 0002:00000028       __imp__GetModuleFileNameA@12 1000b028     kernel32:KERNEL32.dll
 0002:0000002c       __imp__GetModuleHandleA@4  1000b02c     kernel32:KERNEL32.dll
 0002:00000030       __imp__GetModuleHandleExA@12 1000b030     kernel32:KERNEL32.dll
 0002:00000034       __imp__GetProcAddress@8    1000b034     kernel32:KERNEL32.dll
 0002:00000038       __imp__LoadLibraryA@4      1000b038     kernel32:KERNEL32.dll
 0002:0000003c       __imp__LocalFree@4         1000b03c     kernel32:KERNEL32.dll
 0002:00000040       __imp__FormatMessageA@28   1000b040     kernel32:KERNEL32.dll
 0002:00000044       __imp__FindClose@4         1000b044     kernel32:KERNEL32.dll
 0002:00000048       __imp__FindFirstFileA@8    1000b048     kernel32:KERNEL32.dll
 0002:0000004c       __imp__FindNextFileA@8     1000b04c     kernel32:KERNEL32.dll
 0002:00000050       __imp__UnhandledExceptionFilter@4 1000b050     kernel32:KERNEL32.dll
 0002:00000054       __imp__SetUnhandledExceptionFilter@4 1000b054     kernel32:KERNEL32.dll
 0002:00000058       __imp__GetCurrentProcess@0 1000b058     kernel32:KERNEL32.dll
 0002:0000005c       __imp__TerminateProcess@8  1000b05c     kernel32:KERNEL32.dll
 0002:00000060       __imp__IsProcessorFeaturePresent@4 1000b060     kernel32:KERNEL32.dll
 0002:00000064       __imp__GetCurrentProcessId@0 1000b064     kernel32:KERNEL32.dll
 0002:00000068       __imp__GetCurrentThreadId@0 1000b068     kernel32:KERNEL32.dll
 0002:0000006c       __imp__GetSystemTimeAsFileTime@4 1000b06c     kernel32:KERNEL32.dll
 0002:00000070       __imp__DisableThreadLibraryCalls@4 1000b070     kernel32:KERNEL32.dll
 0002:00000074       __imp__InitializeSListHead@4 1000b074     kernel32:KERNEL32.dll
 0002:00000078       \177KERNEL32_NULL_THUNK_DATA 1000b078     kernel32:KERNEL32.dll
 0002:0000007c       __imp__CharNextExA@12      1000b07c     user32:USER32.dll
 0002:00000080       __imp__MessageBoxA@16      1000b080     user32:USER32.dll
 0002:00000084       \177USER32_NULL_THUNK_DATA 1000b084     user32:USER32.dll
 0002:00000088       __imp__memcpy              1000b088     vcruntime:VCRUNTIME140.dll
 0002:0000008c       __imp__strchr              1000b08c     vcruntime:VCRUNTIME140.dll
 0002:00000090       __imp__memset              1000b090     vcruntime:VCRUNTIME140.dll
 0002:00000094       __imp__strrchr             1000b094     vcruntime:VCRUNTIME140.dll
 0002:00000098       __imp__memcmp              1000b098     vcruntime:VCRUNTIME140.dll
 0002:0000009c       __imp__memmove             1000b09c     vcruntime:VCRUNTIME140.dll
 0002:000000a0       __imp____std_type_info_destroy_list 1000b0a0     vcruntime:VCRUNTIME140.dll
 0002:000000a4       __imp___except_handler4_common 1000b0a4     vcruntime:VCRUNTIME140.dll
 0002:000000a8       \177VCRUNTIME140_NULL_THUNK_DATA 1000b0a8     vcruntime:VCRUNTIME140.dll
 0002:000000ac       __imp__mbstowcs            1000b0ac     ucrt:api-ms-win-crt-convert-l1-1-0.dll
 0002:000000b0       \177api-ms-win-crt-convert-l1-1-0_NULL_THUNK_DATA 1000b0b0     ucrt:api-ms-win-crt-convert-l1-1-0.dll
 0002:000000b4       __imp__getenv              1000b0b4     ucrt:api-ms-win-crt-environment-l1-1-0.dll
 0002:000000b8       __imp___putenv             1000b0b8     ucrt:api-ms-win-crt-environment-l1-1-0.dll
 0002:000000b8       __imp__putenv              1000b0b8     ucrt:api-ms-win-crt-environment-l1-1-0.dll
 0002:000000bc       \177api-ms-win-crt-environment-l1-1-0_NULL_THUNK_DATA 1000b0bc     ucrt:api-ms-win-crt-environment-l1-1-0.dll
 0002:000000c0       __imp___wfullpath          1000b0c0     ucrt:api-ms-win-crt-filesystem-l1-1-0.dll
 0002:000000c4       __imp___stat64i32          1000b0c4     ucrt:api-ms-win-crt-filesystem-l1-1-0.dll
 0002:000000c8       __imp___access             1000b0c8     ucrt:api-ms-win-crt-filesystem-l1-1-0.dll
 0002:000000cc       \177api-ms-win-crt-filesystem-l1-1-0_NULL_THUNK_DATA 1000b0cc     ucrt:api-ms-win-crt-filesystem-l1-1-0.dll
 0002:000000d0       __imp__malloc              1000b0d0     ucrt:api-ms-win-crt-heap-l1-1-0.dll
 0002:000000d4       __imp__free                1000b0d4     ucrt:api-ms-win-crt-heap-l1-1-0.dll
 0002:000000d8       __imp__realloc             1000b0d8     ucrt:api-ms-win-crt-heap-l1-1-0.dll
 0002:000000dc       __imp__calloc              1000b0dc     ucrt:api-ms-win-crt-heap-l1-1-0.dll
 0002:000000e0       \177api-ms-win-crt-heap-l1-1-0_NULL_THUNK_DATA 1000b0e0     ucrt:api-ms-win-crt-heap-l1-1-0.dll
 0002:000000e4       __imp___seh_filter_dll     1000b0e4     ucrt:api-ms-win-crt-runtime-l1-1-0.dll
 0002:000000e8       __imp___initterm           1000b0e8     ucrt:api-ms-win-crt-runtime-l1-1-0.dll
 0002:000000ec       __imp___configure_narrow_argv 1000b0ec     ucrt:api-ms-win-crt-runtime-l1-1-0.dll
 0002:000000f0       __imp___initialize_narrow_environment 1000b0f0     ucrt:api-ms-win-crt-runtime-l1-1-0.dll
 0002:000000f4       __imp__perror              1000b0f4     ucrt:api-ms-win-crt-runtime-l1-1-0.dll
 0002:000000f8       __imp__exit                1000b0f8     ucrt:api-ms-win-crt-runtime-l1-1-0.dll
 0002:000000fc       __imp___initialize_onexit_table 1000b0fc     ucrt:api-ms-win-crt-runtime-l1-1-0.dll
 0002:00000100       __imp___getpid             1000b100     ucrt:api-ms-win-crt-runtime-l1-1-0.dll
 0002:00000104       __imp___errno              1000b104     ucrt:api-ms-win-crt-runtime-l1-1-0.dll
 0002:00000108       __imp___cexit              1000b108     ucrt:api-ms-win-crt-runtime-l1-1-0.dll
 0002:0000010c       __imp__strerror            1000b10c     ucrt:api-ms-win-crt-runtime-l1-1-0.dll
 0002:00000110       __imp___initterm_e         1000b110     ucrt:api-ms-win-crt-runtime-l1-1-0.dll
 0002:00000114       __imp___beginthreadex      1000b114     ucrt:api-ms-win-crt-runtime-l1-1-0.dll
 0002:00000118       __imp___execute_onexit_table 1000b118     ucrt:api-ms-win-crt-runtime-l1-1-0.dll
 0002:0000011c       \177api-ms-win-crt-runtime-l1-1-0_NULL_THUNK_DATA 1000b11c     ucrt:api-ms-win-crt-runtime-l1-1-0.dll
 0002:00000120       __imp__close               1000b120     ucrt:api-ms-win-crt-stdio-l1-1-0.dll
 0002:00000120       __imp___close              1000b120     ucrt:api-ms-win-crt-stdio-l1-1-0.dll
 0002:00000124       __imp___read               1000b124     ucrt:api-ms-win-crt-stdio-l1-1-0.dll
 0002:00000124       __imp__read                1000b124     ucrt:api-ms-win-crt-stdio-l1-1-0.dll
 0002:00000128       __imp__fflush              1000b128     ucrt:api-ms-win-crt-stdio-l1-1-0.dll
 0002:0000012c       __imp__fclose              1000b12c     ucrt:api-ms-win-crt-stdio-l1-1-0.dll
 0002:00000130       __imp___open_osfhandle     1000b130     ucrt:api-ms-win-crt-stdio-l1-1-0.dll
 0002:00000134       __imp____stdio_common_vsscanf 1000b134     ucrt:api-ms-win-crt-stdio-l1-1-0.dll
 0002:00000138       __imp____stdio_common_vsprintf 1000b138     ucrt:api-ms-win-crt-stdio-l1-1-0.dll
 0002:0000013c       __imp___lseeki64           1000b13c     ucrt:api-ms-win-crt-stdio-l1-1-0.dll
 0002:00000140       __imp____stdio_common_vfprintf 1000b140     ucrt:api-ms-win-crt-stdio-l1-1-0.dll
 0002:00000144       __imp__fgets               1000b144     ucrt:api-ms-win-crt-stdio-l1-1-0.dll
 0002:00000148       __imp____acrt_iob_func     1000b148     ucrt:api-ms-win-crt-stdio-l1-1-0.dll
 0002:0000014c       __imp__fread               1000b14c     ucrt:api-ms-win-crt-stdio-l1-1-0.dll
 0002:00000150       __imp__fopen               1000b150     ucrt:api-ms-win-crt-stdio-l1-1-0.dll
 0002:00000154       __imp__ferror              1000b154     ucrt:api-ms-win-crt-stdio-l1-1-0.dll
 0002:00000158       __imp__feof                1000b158     ucrt:api-ms-win-crt-stdio-l1-1-0.dll
 0002:0000015c       __imp___open               1000b15c     ucrt:api-ms-win-crt-stdio-l1-1-0.dll
 0002:00000160       \177api-ms-win-crt-stdio-l1-1-0_NULL_THUNK_DATA 1000b160     ucrt:api-ms-win-crt-stdio-l1-1-0.dll
 0002:00000164       __imp__strncmp             1000b164     ucrt:api-ms-win-crt-string-l1-1-0.dll
 0002:00000168       __imp__wcslen              1000b168     ucrt:api-ms-win-crt-string-l1-1-0.dll
 0002:0000016c       __imp__wcscpy              1000b16c     ucrt:api-ms-win-crt-string-l1-1-0.dll
 0002:00000170       __imp__stricmp             1000b170     ucrt:api-ms-win-crt-string-l1-1-0.dll
 0002:00000170       __imp___stricmp            1000b170     ucrt:api-ms-win-crt-string-l1-1-0.dll
 0002:00000174       __imp__strdup              1000b174     ucrt:api-ms-win-crt-string-l1-1-0.dll
 0002:00000174       __imp___strdup             1000b174     ucrt:api-ms-win-crt-string-l1-1-0.dll
 0002:00000178       __imp__strspn              1000b178     ucrt:api-ms-win-crt-string-l1-1-0.dll
 0002:0000017c       __imp__strcspn             1000b17c     ucrt:api-ms-win-crt-string-l1-1-0.dll
 0002:00000180       __imp__strcpy              1000b180     ucrt:api-ms-win-crt-string-l1-1-0.dll
 0002:00000184       __imp__strcat              1000b184     ucrt:api-ms-win-crt-string-l1-1-0.dll
 0002:00000188       __imp__strpbrk             1000b188     ucrt:api-ms-win-crt-string-l1-1-0.dll
 0002:0000018c       __imp__strlen              1000b18c     ucrt:api-ms-win-crt-string-l1-1-0.dll
 0002:00000190       __imp__isspace             1000b190     ucrt:api-ms-win-crt-string-l1-1-0.dll
 0002:00000194       __imp__strcmp              1000b194     ucrt:api-ms-win-crt-string-l1-1-0.dll
 0002:00000198       \177api-ms-win-crt-string-l1-1-0_NULL_THUNK_DATA 1000b198     ucrt:api-ms-win-crt-string-l1-1-0.dll
 0002:0000019c       ___guard_check_icall_fptr  1000b19c     MSVCRT:guard_support.obj
 0002:000001a0       ___xc_a                    1000b1a0     MSVCRT:initializers.obj
 0002:000001a4       ___xc_z                    1000b1a4     MSVCRT:initializers.obj
 0002:000001a8       ___xi_a                    1000b1a8     MSVCRT:initializers.obj
 0002:000001ac       ___xi_z                    1000b1ac     MSVCRT:initializers.obj
 0002:000001b0       ___xp_a                    1000b1b0     MSVCRT:initializers.obj
 0002:000001b4       ___xp_z                    1000b1b4     MSVCRT:initializers.obj
 0002:000001b8       ___xt_a                    1000b1b8     MSVCRT:initializers.obj
 0002:000001bc       ___xt_z                    1000b1bc     MSVCRT:initializers.obj
 0002:000001c0       ??_C@_07NBCGADJA@Unknown@  1000b1c0     args.obj
 0002:000001c8       ??_C@_0L@EOAAECLN@Main?5class@ 1000b1c8     args.obj
 0002:000001d4       ??_C@_08NIAMKNB@JAR?5file@ 1000b1d4     args.obj
 0002:000001e0       ??_C@_06NHPJKFDC@Module@   1000b1e0     args.obj
 0002:000001e8       ??_C@_06CLBDIDBH@Source@   1000b1e8     args.obj
 0002:000001f0       ??_C@_04LEOFD@?9jar@       1000b1f0     args.obj
 0002:000001f8       ??_C@_08HCOMEFAN@?9?9module@ 1000b1f8     args.obj
 0002:00000204       ??_C@_02OAHIOGLE@?9m@      1000b204     args.obj
 0002:00000208       ??_C@_0BB@MIOGFJGG@?9?9disable?9?$EAfiles@ 1000b208     args.obj
 0002:0000021c       ??_C@_0BL@FBFFBAJO@Error?3?5could?5not?5open?5?$GA?$CFs?8@ 1000b21c     args.obj
 0002:00000238       ??_C@_01KDCPPGHE@r@        1000b238     args.obj
 0002:0000023c       ??_C@_0BD@FIJKEMFL@Error?3?5loading?3?5?$CFs@ 1000b23c     args.obj
 0002:00000250       ??_C@_08IOAGGDCI@?9?9source@ 1000b250     args.obj
 0002:0000025c       ??_C@_09IHDACGGH@?9?9dry?9run@ 1000b25c     args.obj
 0002:00000268       ??_C@_02JNAPBCPB@?9h@      1000b268     args.obj
 0002:0000026c       ??_C@_02GIPFNJGC@?9?$DP@   1000b26c     args.obj
 0002:00000270       ??_C@_05DOEHDILL@?9help@   1000b270     args.obj
 0002:00000278       ??_C@_06LMIDBODK@?9?9help@ 1000b278     args.obj
 0002:00000280       ??_C@_02ECEJCEAC@?9X@      1000b280     args.obj
 0002:00000284       ??_C@_0N@LJKGKPCB@?9?9help?9extra@ 1000b284     args.obj
 0002:00000294       ??_C@_08NPLKDBJI@?9version@ 1000b294     args.obj
 0002:000002a0       ??_C@_09GAJKMFCA@?9?9version@ 1000b2a0     args.obj
 0002:000002ac       ??_C@_0N@IILNIMNM@?9fullversion@ 1000b2ac     args.obj
 0002:000002bc       ??_C@_0P@GDNPHBKG@?9?9full?9version@ 1000b2bc     args.obj
 0002:000002cc       ??_C@_0BH@CNAHHPOK@NOTE?3?5Picked?5up?5?$CFs?3?5?$CFs@ 1000b2cc     args.obj
 0002:000002e4       ??_C@_0DC@KPFLGICH@Error?3?5Unmatched?5quote?5in?5envir@ 1000b2e4     args.obj
 0002:00000318       ??_C@_0DL@BPENDAOO@Error?3?5Option?5?$CFs?5is?5not?5allowed@ 1000b318     args.obj
 0002:00000354       ??_C@_0DA@LDDJJBHL@Error?3?5Option?5?$CFs?5is?5not?5allowed@ 1000b354     args.obj
 0002:00000388       ??_C@_0EB@LNOCLEBI@Error?3?5Option?5?$CFs?5in?5?$CFs?5is?5not?5a@ 1000b388     args.obj
 0002:000003cc       ??_C@_0DG@JOFJKKPC@Error?3?5Option?5?$CFs?5in?5?$CFs?5is?5not?5a@ 1000b3cc     args.obj
 0002:00000404       ??_C@_0DM@EJAEKOHO@Error?3?5Cannot?5specify?5main?5clas@ 1000b404     args.obj
 0002:00000440       ??_C@_0DB@OCKOCINB@Error?3?5Cannot?5specify?5main?5clas@ 1000b440     args.obj
 0002:00000474       ??_C@_0BB@JPFIPKCP@JDK_JAVA_OPTIONS@ 1000b474     cmdtoargs.obj
 0002:00000488       ??_C@_0BF@FJHGBKOC@_JAVA_LAUNCHER_DEBUG@ 1000b488     cmdtoargs.obj
 0002:000004a0       ??_C@_0O@GCGKPAG@_JAVA_OPTIONS@ 1000b4a0     cmdtoargs.obj
 0002:000004b0       ??_C@_0BO@ECPMAOGG@invalid?5distance?5too?5far?5back@ 1000b4b0     inffast.obj
 0002:000004d0       ??_C@_0BG@LBKINIKP@invalid?5distance?5code@ 1000b4d0     inffast.obj
 0002:000004e8       ??_C@_0BM@FFFLPBBC@invalid?5literal?1length?5code@ 1000b4e8     inffast.obj
 0002:00000db0       ??_C@_0BH@LIBMMIGA@incorrect?5header?5check@ 1000bdb0     inflate.obj
 0002:00000dc8       ??_C@_0BL@IHKGDAEE@unknown?5compression?5method@ 1000bdc8     inflate.obj
 0002:00000de4       ??_C@_0BE@EMOGCLGO@invalid?5window?5size@ 1000bde4     inflate.obj
 0002:00000df8       ??_C@_0BJ@BLBBCOMO@unknown?5header?5flags?5set@ 1000bdf8     inflate.obj
 0002:00000e14       ??_C@_0BE@GONKLEPM@header?5crc?5mismatch@ 1000be14     inflate.obj
 0002:00000e28       ??_C@_0BD@PJCBIDD@invalid?5block?5type@ 1000be28     inflate.obj
 0002:00000e3c       ??_C@_0BN@LGAADGOK@invalid?5stored?5block?5lengths@ 1000be3c     inflate.obj
 0002:00000e5c       ??_C@_0CE@GMIGFPBB@too?5many?5length?5or?5distance?5sym@ 1000be5c     inflate.obj
 0002:00000e80       ??_C@_0BJ@HDEPPGOH@invalid?5code?5lengths?5set@ 1000be80     inflate.obj
 0002:00000e9c       ??_C@_0BK@BMMPFBBH@invalid?5bit?5length?5repeat@ 1000be9c     inflate.obj
 0002:00000eb8       ??_C@_0CF@DGDMADCD@invalid?5code?5?9?9?5missing?5end?9of?9@ 1000beb8     inflate.obj
 0002:00000ee0       ??_C@_0BM@IIMGAINC@invalid?5literal?1lengths?5set@ 1000bee0     inflate.obj
 0002:00000efc       ??_C@_0BG@GMDFCBGP@invalid?5distances?5set@ 1000befc     inflate.obj
 0002:00000f14       ??_C@_0BF@MEIGEHBE@incorrect?5data?5check@ 1000bf14     inflate.obj
 0002:00000f2c       ??_C@_0BH@FGKKJGOC@incorrect?5length?5check@ 1000bf2c     inflate.obj
 0002:00000f48       _inflate_copyright         1000bf48     inftrees.obj
 0002:00001078       ??_C@_0L@FLLOCCHD@NMT_LEVEL_@ 1000c078     java.obj
 0002:000010bc       ??_C@_02OJDBNLEE@?5?7@     1000c0bc     java.obj
 0002:000010c0       ??_C@_0M@GMLNOKOP@Java?5args?3?6@ 1000c0c0     java.obj
 0002:000010cc       ??_C@_0BA@CGOOFFNP@jargv?$FL?$CFd?$FN?5?$DN?5?$CFs?6@ 1000c0cc     java.obj
 0002:000010dc       ??_C@_0BE@OFPFKAIO@Command?5line?5args?3?6@ 1000c0dc     java.obj
 0002:000010f0       ??_C@_0P@NAHECKMG@argv?$FL?$CFd?$FN?5?$DN?5?$CFs?6@ 1000c0f0     java.obj
 0002:00001100       ??_C@_0BO@JELEMDBE@?9Dsun?4java?4launcher?4diag?$DNtrue@ 1000c100     java.obj
 0002:00001120       ??_C@_0CB@IBPGMCMH@?$CFld?5micro?5seconds?5to?5LoadJavaVM@ 1000c120     java.obj
 0002:00001144       ??_C@_09GEOACDML@CLASSPATH@ 1000c144     java.obj
 0002:00001150       ??_C@_0GM@ELCKKLGK@Error?3?5Could?5not?5create?5the?5Jav@ 1000c150     java.obj
 0002:000011c0       ??_C@_0HD@PPKHMHGL@Error?3?5Could?5not?5detach?5main?5th@ 1000c1c0     java.obj
 0002:00001234       ??_C@_0CE@ODMOBDNM@?$CFld?5micro?5seconds?5to?5Initialize@ 1000c234     java.obj
 0002:00001258       ??_C@_0M@JMGIBICN@?$CFs?5is?5?8?$CFs?8?6@ 1000c258     java.obj
 0002:00001264       ??_C@_0BC@IKMDOBPK@App?8s?5argc?5is?5?$CFd?6@ 1000c264     java.obj
 0002:00001278       ??_C@_0BG@EAAKBDAJ@?5?5?5?5argv?$FL?$CF2d?$FN?5?$DN?5?8?$CFs?8?6@ 1000c278     java.obj
 0002:00001290       ??_C@_0EO@KGGGJHNP@Error?3?5A?5JNI?5error?5has?5occurred@ 1000c290     java.obj
 0002:000012e0       ??_C@_0BH@IALIHDHM@?$CI?$FLLjava?1lang?1String?$DL?$CJV@ 1000c2e0     java.obj
 0002:000012f8       ??_C@_04GHJNJNPO@main@     1000c2f8     java.obj
 0002:00001300       ??_C@_0L@JBBEAFHG@?9classpath@ 1000c300     java.obj
 0002:0000130c       ??_C@_03OJENFLIP@?9cp@     1000c30c     java.obj
 0002:00001310       ??_C@_0N@LELNCGH@?9?9class?9path@ 1000c310     java.obj
 0002:00001320       ??_C@_0BC@ILEAKADP@?9?9describe?9module@ 1000c320     java.obj
 0002:00001334       ??_C@_02DBLKFNPN@?9d@      1000c334     java.obj
 0002:00001338       ??_C@_0O@NGANBJGM@?9?9module?9path@ 1000c338     java.obj
 0002:00001348       ??_C@_02BPBEIKKI@?9p@      1000c348     java.obj
 0002:0000134c       ??_C@_0BG@ONLDFKAD@?9?9upgrade?9module?9path@ 1000c34c     java.obj
 0002:00001364       ??_C@_0O@PHHJGBMD@?9?9add?9modules@ 1000c364     java.obj
 0002:00001374       ??_C@_0BA@OIHFEKDD@?9?9limit?9modules@ 1000c374     java.obj
 0002:00001384       ??_C@_0O@JJNAPOHD@?9?9add?9exports@ 1000c384     java.obj
 0002:00001394       ??_C@_0M@MAAOPOMD@?9?9add?9opens@ 1000c394     java.obj
 0002:000013a0       ??_C@_0M@FFLDOFPF@?9?9add?9reads@ 1000c3a0     java.obj
 0002:000013ac       ??_C@_0P@KEEOJCPM@?9?9patch?9module@ 1000c3ac     java.obj
 0002:000013bc       ??_C@_0P@CODKGINE@?9?9module?9path?$DN@ 1000c3bc     java.obj
 0002:000013cc       ??_C@_0BH@PDAMKKFO@?9?9upgrade?9module?9path?$DN@ 1000c3cc     java.obj
 0002:000013e4       ??_C@_0P@GIHCKCNF@?9?9add?9modules?$DN@ 1000c3e4     java.obj
 0002:000013f4       ??_C@_0BB@NFNAFMOC@?9?9limit?9modules?$DN@ 1000c3f4     java.obj
 0002:00001408       ??_C@_0P@KDHNLIMG@?9?9add?9exports?$DN@ 1000c408     java.obj
 0002:00001418       ??_C@_0N@KHGKPNMI@?9?9add?9reads?$DN@ 1000c418     java.obj
 0002:00001428       ??_C@_0BA@NOEHLIBL@?9?9patch?9module?$DN@ 1000c428     java.obj
 0002:00001438       ??_C@_0CO@PJHOEEID@Error?3?5Option?5?$CFs?5is?5not?5allowed@ 1000c438     java.obj
 0002:00001468       ??_C@_05PBJILJE@?4java@    1000c468     java.obj
 0002:00001470       ??_C@_0BB@BIGIFKOD@JDK_ALTERNATE_VM@ 1000c470     java.obj
 0002:00001484       ??_C@_0L@MNOMOABD@?9XXaltjvm?$DN@ 1000c484     java.obj
 0002:00001490       ??_C@_0N@IHBJGDGH@?9J?9XXaltjvm?$DN@ 1000c490     java.obj
 0002:000014a0       ??_C@_0BA@ENLNODBJ@Default?5VM?3?5?$CFs?6@ 1000c4a0     java.obj
 0002:000014b0       ??_C@_0DC@GMKJBLDL@Error?3?5Corrupt?5jvm?4cfg?5file?$DL?5cy@ 1000c4b0     java.obj
 0002:000014e4       ??_C@_05MBDEGLCK@ERROR@    1000c4e4     java.obj
 0002:000014ec       ??_C@_0CF@EHKDFPIN@Error?3?5Unable?5to?5resolve?5VM?5ali@ 1000c4ec     java.obj
 0002:00001514       ??_C@_0DB@ICJLIDMC@Warning?3?5?$CFs?5VM?5not?5supported?$DL?5?$CF@ 1000c514     java.obj
 0002:00001548       ??_C@_0BL@ICJEGBLP@Error?3?5?$CFs?5VM?5not?5supported@ 1000c548     java.obj
 0002:00001564       ??_C@_0BK@KPPPPIMG@?9XX?3NativeMemoryTracking?$DN@ 1000c564     java.obj
 0002:00001580       ??_C@_07PFMNENFI@?$CFs?$CFd?$DN?$CFs@ 1000c580     java.obj
 0002:00001588       ??_C@_04HGGBINEM@?$CFs?$CFd@ 1000c588     java.obj
 0002:00001590       ??_C@_0DE@KEMGKHHI@TRACER_MARKER?3?5NativeMemoryTrac@ 1000c590     java.obj
 0002:000015c4       ??_C@_0DE@KHHPGILD@TRACER_MARKER?3?5NativeMemoryTrac@ 1000c5c4     java.obj
 0002:000015f8       ??_C@_0DD@JGMKIPCJ@TRACER_MARKER?3?5NativeMemoryTrac@ 1000c5f8     java.obj
 0002:0000162c       ??_C@_05LLAMLEHD@?$CFI64d@ 1000c62c     java.obj
 0002:00001634       ??_C@_04FMJADICG@?9Xss@    1000c634     java.obj
 0002:0000163c       ??_C@_04KJNMGPJH@?9Xmx@    1000c63c     java.obj
 0002:00001644       ??_C@_04EKCILGFM@?9Xms@    1000c644     java.obj
 0002:0000164c       ??_C@_0BC@LDDPFIIH@_JAVA_VERSION_SET@ 1000c64c     java.obj
 0002:00001660       ??_C@_09NLKCHPDO@?9version?3@ 1000c660     java.obj
 0002:00001670       ??_C@_0LE@PIKCPCAG@Error?3?5Specifying?5an?5alternate?5@ 1000c670     java.obj
 0002:00001724       ??_C@_0BF@BOPFKIEC@?9jre?9restrict?9search@ 1000c724     java.obj
 0002:00001740       ??_C@_0JM@NGABGLOK@Error?3?5Specifying?5an?5alternate?5@ 1000c740     java.obj
 0002:000017dc       ??_C@_0BI@PDBPIFBH@?9jre?9no?9restrict?9search@ 1000c7dc     java.obj
 0002:000017f4       ??_C@_0BJ@MCNGENOM@?9Djava?4awt?4headless?$DNtrue@ 1000c7f4     java.obj
 0002:00001810       ??_C@_0BF@CMFGICHD@?9Djava?4awt?4headless?$DN@ 1000c810     java.obj
 0002:00001828       ??_C@_08GFHMBCLC@?9splash?3@ 1000c828     java.obj
 0002:00001834       ??_C@_0CD@DBKPDEJE@Error?3?5Unable?5to?5access?5jarfile@ 1000c834     java.obj
 0002:00001858       ??_C@_0CF@JOEJCGOC@Error?3?5Invalid?5or?5corrupt?5jarfi@ 1000c858     java.obj
 0002:00001880       ??_C@_0BD@NDCPPKLD@_JAVA_SPLASH_FILE?$DN@ 1000c880     java.obj
 0002:00001894       ??_C@_0BC@FAHMLMBM@_JAVA_SPLASH_JAR?$DN@ 1000c894     java.obj
 0002:000018a8       ??_C@_02BAABKJLB@?9?9@     1000c8a8     java.obj
 0002:000018ac       ??_C@_0BD@NMAFCFCD@?9?9describe?9module?$DN@ 1000c8ac     java.obj
 0002:000018c0       ??_C@_09BECLNIEG@?9?9module?$DN@ 1000c8c0     java.obj
 0002:000018cc       ??_C@_0O@LJDFPHJH@?9?9class?9path?$DN@ 1000c8cc     java.obj
 0002:000018dc       ??_C@_09FPNDOGCH@?9?9source?$DN@ 1000c8dc     java.obj
 0002:000018e8       ??_C@_0CK@JHECGGGO@Error?3?5?$CFs?5requires?5jar?5file?5spe@ 1000c8e8     java.obj
 0002:00001914       ??_C@_0BP@KOJLKEHJ@Error?3?5?$CFs?5requires?5module?5name@ 1000c914     java.obj
 0002:00001934       ??_C@_0CC@GJJMCLCA@Error?3?5?$CFs?5requires?5source?5versi@ 1000c934     java.obj
 0002:00001958       ??_C@_0BN@MGNCCAPH@?9Djdk?4internal?4javac?4source?$DN@ 1000c958     java.obj
 0002:00001978       ??_C@_04HDOCAJNK@?$CFs?$CFs@ 1000c978     java.obj
 0002:00001980       ??_C@_0CM@DPCHNCBN@Error?3?5?$CFs?5requires?5class?5path?5s@ 1000c980     java.obj
 0002:000019ac       ??_C@_0P@EDKODJAB@?9?9list?9modules@ 1000c9ac     java.obj
 0002:000019bc       ??_C@_0BI@BOPIBLJA@?9?9show?9resolved?9modules@ 1000c9bc     java.obj
 0002:000019d4       ??_C@_0BD@DDNDIFKN@?9?9validate?9modules@ 1000c9d4     java.obj
 0002:000019e8       ??_C@_0BN@ENOFGBKM@?9Djdk?4module?4validation?$DNtrue@ 1000c9e8     java.obj
 0002:00001a08       ??_C@_0CN@EKOIGANM@Error?3?5?$CFs?5requires?5module?5path?5@ 1000ca08     java.obj
 0002:00001a38       ??_C@_0CL@NJCCMCJP@Error?3?5?$CFs?5requires?5modules?5to?5b@ 1000ca38     java.obj
 0002:00001a64       ??_C@_0N@LMMGPIFD@?9showversion@ 1000ca64     java.obj
 0002:00001a74       ??_C@_0P@BOOMJEGD@?9?9show?9version@ 1000ca74     java.obj
 0002:00001a84       ??_C@_0P@OLHNJJJN@?9XshowSettings@ 1000ca84     java.obj
 0002:00001a94       ??_C@_0BA@KLPMEMBJ@?9XshowSettings?3@ 1000ca94     java.obj
 0002:00001aa4       ??_C@_06GFBBMHDE@?9Xdiag@  1000caa4     java.obj
 0002:00001aac       ??_C@_0BJ@HFDHICEA@?9?9show?9module?9resolution@ 1000caac     java.obj
 0002:00001ac8       ??_C@_0CH@PGFFCLHP@?9Djdk?4module?4showModuleResoluti@ 1000cac8     java.obj
 0002:00001af0       ??_C@_0BF@CGIIANBK@?$CFs?5full?5version?5?$CC?$CFs?$CC@ 1000caf0     java.obj
 0002:00001b08       ??_C@_05DNIIFBMG@?$CFs?5?$CFs@ 1000cb08     java.obj
 0002:00001b10       ??_C@_0L@IOOPLDLG@?9verbosegc@ 1000cb10     java.obj
 0002:00001b1c       ??_C@_0M@FCDCLOMN@?9verbose?3gc@ 1000cb1c     java.obj
 0002:00001b28       ??_C@_02HLHIEPKM@?9t@      1000cb28     java.obj
 0002:00001b2c       ??_C@_03KFBPJEPK@?9Xt@     1000cb2c     java.obj
 0002:00001b30       ??_C@_03PEIICGG@?9tm@      1000cb30     java.obj
 0002:00001b34       ??_C@_04INJOBBHM@?9Xtm@    1000cb34     java.obj
 0002:00001b3c       ??_C@_06OHOHKFPP@?9debug@  1000cb3c     java.obj
 0002:00001b44       ??_C@_07MDIKCNOD@?9Xdebug@ 1000cb44     java.obj
 0002:00001b4c       ??_C@_0L@IAOONLOP@?9noclassgc@ 1000cb4c     java.obj
 0002:00001b58       ??_C@_0M@JJFHIIML@?9Xnoclassgc@ 1000cb58     java.obj
 0002:00001b64       ??_C@_08EAEOLGAG@?9Xfuture@ 1000cb64     java.obj
 0002:00001b70       ??_C@_0N@CKMDLKDL@?9Xverify?3all@ 1000cb70     java.obj
 0002:00001b80       ??_C@_07FILEFCOC@?9verify@ 1000cb80     java.obj
 0002:00001b88       ??_C@_0O@IDLLNEML@?9verifyremote@ 1000cb88     java.obj
 0002:00001b98       ??_C@_0BA@FABHJJHD@?9Xverify?3remote@ 1000cb98     java.obj
 0002:00001ba8       ??_C@_09JLKGPCDL@?9noverify@ 1000cba8     java.obj
 0002:00001bb4       ??_C@_0O@DKMKFJCN@?9Xverify?3none@ 1000cbb4     java.obj
 0002:00001bc4       ??_C@_03NOEGKLDM@?9ss@     1000cbc4     java.obj
 0002:00001bc8       ??_C@_04DBGMPIDO@?9oss@    1000cbc8     java.obj
 0002:00001bd0       ??_C@_03MIPOCFEG@?9ms@     1000cbd0     java.obj
 0002:00001bd4       ??_C@_03CLAKPMIN@?9mx@     1000cbd4     java.obj
 0002:00001bd8       ??_C@_04DEKBGKCE@?9X?$CFs@ 1000cbd8     java.obj
 0002:00001be0       ??_C@_0N@OIJOAPMB@?9checksource@ 1000cbe0     java.obj
 0002:00001bf0       ??_C@_03MCGAAIEM@?9cs@     1000cbf0     java.obj
 0002:00001bf4       ??_C@_0L@HELBLEOP@?9noasyncgc@ 1000cbf4     java.obj
 0002:00001c00       ??_C@_0CL@CAKBCILK@Warning?3?5?$CFs?5option?5is?5no?5longer@ 1000cc00     java.obj
 0002:00001c2c       ??_C@_0BD@HCEIMOC@?9Djava?4class?4path?$DN@ 1000cc2c     java.obj
 0002:00001c40       ??_C@_01LFCBOECM@?4@       1000cc40     java.obj
 0002:00001c44       ??_C@_0BK@NCKACBAA@?9?9add?9modules?$DNALL?9DEFAULT@ 1000cc44     java.obj
 0002:00001c60       ??_C@_0CP@EGLKGJHA@jdk?4compiler?1com?4sun?4tools?4java@ 1000cc60     java.obj
 0002:00001c90       ??_C@_0BC@JGENKKKB@JavaVM?5args?3?6?5?5?5?5@ 1000cc90     java.obj
 0002:00001ca4       ??_C@_0BC@FPGFOMNN@version?50x?$CF08lx?0?5@ 1000cca4     java.obj
 0002:00001cb8       ??_C@_08JPIMBKG@JNI_TRUE@  1000ccb8     java.obj
 0002:00001cc4       ??_C@_09OOFGMMEJ@JNI_FALSE@ 1000ccc4     java.obj
 0002:00001cd0       ??_C@_0BL@KOPLOMOC@ignoreUnrecognized?5is?5?$CFs?0?5@ 1000ccd0     java.obj
 0002:00001cec       ??_C@_0BB@MHDPODII@nOptions?5is?5?$CFld?6@ 1000ccec     java.obj
 0002:00001d00       ??_C@_0BI@DAIGOBCB@?5?5?5?5option?$FL?$CF2d?$FN?5?$DN?5?8?$CFs?8?6@ 1000cd00     java.obj
 0002:00001d18       ??_C@_0BM@GGJONNLD@sun?1launcher?1LauncherHelper@ 1000cd18     java.obj
 0002:00001d34       ??_C@_0BI@DIGBKJNJ@?$CIZ?$FLB?$CJLjava?1lang?1String?$DL@ 1000cd34     java.obj
 0002:00001d4c       ??_C@_0BD@KFHODOP@makePlatformString@ 1000cd4c     java.obj
 0002:00001d60       ??_C@_0BB@FLFAIHG@java?1lang?1String@ 1000cd60     java.obj
 0002:00001d74       ??_C@_0CI@BKCMKGDB@?$CIZILjava?1lang?1String?$DL?$CJLjava?1lan@ 1000cd74     java.obj
 0002:00001d9c       ??_C@_0BB@FFCCDEMN@checkAndLoadMain@ 1000cd9c     java.obj
 0002:00001db0       ??_C@_0CG@FBCAJICK@?$CFld?5micro?5seconds?5to?5load?5main?5@ 1000cdb0     java.obj
 0002:00001dd8       ??_C@_0M@PAPGNNMB@?9?9?9?9?$CFs?9?9?9?9?6@ 1000cdd8     java.obj
 0002:00001de4       ??_C@_0BE@IIFEGCLG@?$CI?$CJLjava?1lang?1Class?$DL@ 1000cde4     java.obj
 0002:00001df8       ??_C@_0BE@JCLPIBOC@getApplicationClass@ 1000cdf8     java.obj
 0002:00001e0c       ??_C@_0DI@DPHDCKMH@Error?3?5The?5?9J?5option?5should?5not@ 1000ce0c     java.obj
 0002:00001e44       ??_C@_0BE@EHGMLIJH@?9Denv?4class?4path?$DN?$CFs@ 1000ce44     java.obj
 0002:00001e58       ??_C@_0CN@LAMKHMKA@Error?3?5Could?5not?5determine?5appl@ 1000ce58     java.obj
 0002:00001e88       ??_C@_0BG@FKBCOFMO@?9Dapplication?4home?$DN?$CFs@ 1000ce88     java.obj
 0002:00001ea0       ??_C@_0BE@NJODCGLC@?9Dsun?4java?4command?$DN@ 1000cea0     java.obj
 0002:00001eb4       ??_C@_01CLKCMJKC@?5@       1000ceb4     java.obj
 0002:00001eb8       ??_C@_0CB@JGILPBEK@?9Dsun?4java?4launcher?$DNSUN_STANDAR@ 1000ceb8     java.obj
 0002:00001edc       ??_C@_0BH@KLEFIFFD@java?1lang?1VersionProps@ 1000cedc     java.obj
 0002:00001ef4       ??_C@_04LHKBAEFM@?$CIZ?$CJV@ 1000cef4     java.obj
 0002:00001efc       ??_C@_07BKGNKEBM@println@  1000cefc     java.obj
 0002:00001f04       ??_C@_05IJDJACGD@print@    1000cf04     java.obj
 0002:00001f0c       ??_C@_0BK@DNGMCIKC@?$CIZLjava?1lang?1String?$DLJJJ?$CJV@ 1000cf0c     java.obj
 0002:00001f28       ??_C@_0N@FDEDEFMB@showSettings@ 1000cf28     java.obj
 0002:00001f38       ??_C@_03GAEACAIP@?$CI?$CJV@ 1000cf38     java.obj
 0002:00001f3c       ??_C@_0BE@HNHCKAIA@showResolvedModules@ 1000cf3c     java.obj
 0002:00001f50       ??_C@_0M@GEBFLOGA@listModules@ 1000cf50     java.obj
 0002:00001f5c       ??_C@_0BG@IKDDPPGD@?$CILjava?1lang?1String?$DL?$CJV@ 1000cf5c     java.obj
 0002:00001f74       ??_C@_0P@GEKKNFKI@describeModule@ 1000cf74     java.obj
 0002:00001f84       ??_C@_0BD@HPNJGMKF@printXUsageMessage@ 1000cf84     java.obj
 0002:00001f98       ??_C@_0BA@KCDLFDGO@initHelpMessage@ 1000cf98     java.obj
 0002:00001fa8       ??_C@_0CI@HEGLGDKJ@?$CILjava?1lang?1String?$DLLjava?1lang?1S@ 1000cfa8     java.obj
 0002:00001fd0       ??_C@_0BG@DGHNKDKK@appendVmSelectMessage@ 1000cfd0     java.obj
 0002:00001fe8       ??_C@_0BH@EGFKIDIP@appendVmSynonymMessage@ 1000cfe8     java.obj
 0002:00002000       ??_C@_0BB@KBOLJHAM@printHelpMessage@ 1000d000     java.obj
 0002:00002014       ??_C@_0CJ@IIPHEFLM@Warning?3?5No?5leading?5?9?5on?5line?5?$CF@ 1000d014     java.obj
 0002:00002040       ??_C@_0CM@HIKCBBNP@Warning?3?5Missing?5VM?5type?5on?5lin@ 1000d040     java.obj
 0002:0000206c       ??_C@_05IBPFAAO@KNOWN@     1000d06c     java.obj
 0002:00002074       ??_C@_0L@PPNPEEBD@ALIASED_TO@ 1000d074     java.obj
 0002:00002080       ??_C@_04JBIELMDE@WARN@     1000d080     java.obj
 0002:00002088       ??_C@_06GHNPMFCC@IGNORE@   1000d088     java.obj
 0002:00002090       ??_C@_0BA@GPBHNCNO@IF_SERVER_CLASS@ 1000d090     java.obj
 0002:000020a0       ??_C@_0CM@FGNACLCO@Warning?3?5Unknown?5VM?5type?5on?5lin@ 1000d0a0     java.obj
 0002:000020cc       ??_C@_0BG@IFIDBPPB@jvm?4cfg?$FL?$CFd?$FN?5?$DN?5?9?$DO?$CFs?$DM?9?6@ 1000d0cc     java.obj
 0002:000020e4       ??_C@_0O@COGEDILL@VM_ALIASED_TO@ 1000d0e4     java.obj
 0002:000020f4       ??_C@_0CF@IFGPMOPD@?5?5?5?5name?3?5?$CFs?5?5vmType?3?5?$CFs?5?5alias@ 1000d0f4     java.obj
 0002:0000211c       ??_C@_0CE@ELPMGLDL@?$CFld?5micro?5seconds?5to?5parse?5jvm?4@ 1000d11c     java.obj
 0002:00002140       ??_C@_02DKLNFENB@?9J@      1000d140     java.obj
 0002:00002144       ??_C@_0BB@CBKFGMGB@_JAVA_SPLASH_JAR@ 1000d144     java.obj
 0002:00002158       ??_C@_0BC@KBGGAEHG@_JAVA_SPLASH_FILE@ 1000d158     java.obj
 0002:0000216c       ??_C@_0BB@PNLKJHCD@Launcher?5state?3?6@ 1000d16c     java.obj
 0002:00002180       ??_C@_0CC@OLAJMMDM@?7First?5application?5arg?5index?3?5?$CF@ 1000d180     java.obj
 0002:000021a4       ??_C@_02LIELOMNJ@on@       1000d1a4     java.obj
 0002:000021a8       ??_C@_03MCADLMAF@off@      1000d1a8     java.obj
 0002:000021ac       ??_C@_0L@MIIHLGHH@?7debug?3?$CFs?6@ 1000d1ac     java.obj
 0002:000021b8       ??_C@_0N@GJJJEEHN@?7javargs?3?$CFs?6@ 1000d1b8     java.obj
 0002:000021c8       ??_C@_0BC@PEOMGKPB@?7program?5name?3?$CFs?6@ 1000d1c8     java.obj
 0002:000021dc       ??_C@_0BD@OJIEGNIP@?7launcher?5name?3?$CFs?6@ 1000d1dc     java.obj
 0002:000021f0       ??_C@_0L@ODBEFCFP@?7javaw?3?$CFs?6@ 1000d1f0     java.obj
 0002:000021fc       ??_C@_0BB@LLCLOLLP@?7fullversion?3?$CFs?6@ 1000d1fc     java.obj
 0002:00002210       ??_C@_01EEMJAFIK@?6@       1000d210     java.obj
 0002:00002214       ??_C@_0BG@JDMBLFEN@?2bin?2splashscreen?4dll@ 1000d214     java_md.obj
 0002:0000222c       ??_C@_04LOAJBDKD@true@     1000d22c     java_md.obj
 0002:00002234       ??_C@_05LAPONLG@false@     1000d234     java_md.obj
 0002:0000223c       ??_C@_0DD@KOHGIEIN@Error?3?5Could?5not?5find?5Java?5SE?5R@ 1000d23c     java_md.obj
 0002:00002270       ??_C@_01KICIPPFI@?2@       1000d270     java_md.obj
 0002:00002274       ??_C@_0BB@DFNCCKIJ@?$CFs?$CFslib?$CFsjvm?4cfg@ 1000d274     java_md.obj
 0002:00002288       ??_C@_0DG@EBKNCNED@Error?3?5no?5known?5VMs?4?5?$CIcheck?5for@ 1000d288     java_md.obj
 0002:000022c0       ??_C@_0CF@EOPDIDEN@Error?3?5could?5not?5determine?5JVM?5@ 1000d2c0     java_md.obj
 0002:000022e8       ??_C@_0GO@EHNKANIL@Error?3?5missing?5?$GA?$CFs?8?5JVM?5at?5?$GA?$CFs?8@ 1000d2e8     java_md.obj
 0002:00002358       ??_C@_0BB@JFPKNOOA@?9Dsun?4awt?4warmup@ 1000d358     java_md.obj
 0002:0000236c       ??_C@_0BF@NJKIMEMJ@?9Dsun?4java2d?4noddraw@ 1000d36c     java_md.obj
 0002:00002384       ??_C@_0BB@NOIMNAMG@?9Dsun?4java2d?4d3d@ 1000d384     java_md.obj
 0002:00002398       ??_C@_0BE@BJJGJMIO@?9Dsun?4java2d?4opengl@ 1000d398     java_md.obj
 0002:000023ac       ??_C@_05MEOKPOAG@?2bin?2@  1000d3ac     java_md.obj
 0002:000023b4       ??_C@_0BB@LMCDEFHL@vcruntime140?4dll@ 1000d3b4     java_md.obj
 0002:000023c8       ??_C@_0DF@CLDFKAFM@Error?3?5Path?5length?5exceeds?5maxi@ 1000d3c8     java_md.obj
 0002:00002400       ??_C@_0BG@HMMNHEMF@?2bin?2vcruntime140?4dll@ 1000d400     java_md.obj
 0002:00002418       ??_C@_0BA@ICKGDIKE@CRT?5path?5is?5?$CFs?6@ 1000d418     java_md.obj
 0002:00002428       ??_C@_0N@GFGFIGJO@msvcp140?4dll@ 1000d428     java_md.obj
 0002:00002438       ??_C@_0BC@GEINBJJF@?2bin?2msvcp140?4dll@ 1000d438     java_md.obj
 0002:0000244c       ??_C@_0BA@ENEJLCMI@PRT?5path?5is?5?$CFs?6@ 1000d44c     java_md.obj
 0002:0000245c       ??_C@_0BA@MFAPGPPP@?$CFs?2bin?2java?4dll@ 1000d45c     java_md.obj
 0002:0000246c       ??_C@_0BA@KEGAOLGA@JRE?5path?5is?5?$CFs?6@ 1000d46c     java_md.obj
 0002:0000247c       ??_C@_0CG@KCIKNEAK@Insufficient?5space?5to?5store?5JRE@ 1000d47c     java_md.obj
 0002:000024a4       ??_C@_0BE@FGKJLOCF@?$CFs?2jre?2bin?2java?4dll@ 1000d4a4     java_md.obj
 0002:000024b8       ??_C@_04NPFKBOJD@?2jre@    1000d4b8     java_md.obj
 0002:000024c0       ??_C@_0BP@GFBADFON@Error?3?5could?5not?5find?5java?4dll@ 1000d4c0     java_md.obj
 0002:000024e0       ??_C@_0L@NCGCEDEH@?$CFs?2jvm?4dll@ 1000d4e0     java_md.obj
 0002:000024ec       ??_C@_0BC@DKEACPBC@?$CFs?2bin?2?$CFs?2jvm?4dll@ 1000d4ec     java_md.obj
 0002:00002500       ??_C@_0BA@BNEFJADF@JVM?5path?5is?5?$CFs?6@ 1000d500     java_md.obj
 0002:00002510       ??_C@_0BB@IDHJDMHA@JNI_CreateJavaVM@ 1000d510     java_md.obj
 0002:00002524       ??_C@_0BN@LEMGLGLC@JNI_GetDefaultJavaVMInitArgs@ 1000d524     java_md.obj
 0002:00002544       ??_C@_0CI@NEHNFCJI@Error?3?5can?8t?5find?5JNI?5interface@ 1000d544     java_md.obj
 0002:0000256c       ??_C@_19MJCDBCKE@?$AA?2?$AA?2?$AA?$DP?$AA?2@ 1000d56c     java_md.obj
 0002:00002578       ??_C@_0BO@HBHLOLEF@Java?5Virtual?5Machine?5Launcher@ 1000d578     java_md.obj
 0002:00002596       ??_C@_00CNPNBAHC@@         1000d596     java_md.obj
 0002:00002598       ??_C@_02DKCKIIND@?$CFs@    1000d598     java_md.obj
 0002:0000259c       ??_C@_0BP@HLKODNMI@A?5Java?5Exception?5has?5occurred?4@ 1000d59c     java_md.obj
 0002:000025bc       ??_C@_01NEMOKFLO@?$DN@     1000d5bc     java_md.obj
 0002:000025c0       ??_C@_07JFLIEEAK@J2D_D3D@  1000d5c0     java_md.obj
 0002:000025c8       ??_C@_0BA@GGNAPKCP@J2D_D3D_PRELOAD@ 1000d5c8     java_md.obj
 0002:000025d8       ??_C@_0L@HNPMBHIG@preloadD3D@ 1000d5d8     java_md.obj
 0002:000025e4       ??_C@_07KCBEICKO@jvm?4dll@ 1000d5e4     java_md.obj
 0002:000025ec       ??_C@_0BM@GLGHANGM@JVM_FindClassFromBootLoader@ 1000d5ec     java_md.obj
 0002:00002608       ??_C@_0BA@MPLLCPDB@?2bin?2verify?4dll@ 1000d608     java_md.obj
 0002:00002618       ??_C@_0O@ICEIELND@?2bin?2java?4dll@ 1000d618     java_md.obj
 0002:00002628       ??_C@_0N@DAAOANPF@?2bin?2awt?4dll@ 1000d628     java_md.obj
 0002:00002638       ??_C@_0M@MLICCBOD@preloadStop@ 1000d638     java_md.obj
 0002:00002644       ??_C@_0DG@HDGLDAO@Warning?3?5app?5args?5is?5larger?5tha@ 1000d644     java_md.obj
 0002:0000267c       ??_C@_0BK@KGACHCN@passing?5arguments?5as?9is?4?6@ 1000d67c     java_md.obj
 0002:00002698       ??_C@_0BO@HHGOPAAH@AppArgIndex?3?5?$CFd?5points?5to?5?$CFs?6@ 1000d698     java_md.obj
 0002:000026b8       ??_C@_0CO@EBEGCMMO@Warning?3?5app?5args?5count?5doesn?8t@ 1000d6b8     java_md.obj
 0002:000026e8       ??_C@_04CDPLFOEF@?$CFc?$CFs@ 1000d6e8     java_md.obj
 0002:000026f0       ??_C@_03OFAPEBGM@?$CFs?6@  1000d6f0     java_md.obj
 0002:000026f4       ??_C@_0CJ@HEGLPLDP@?$CI?$FLLjava?1lang?1String?$DL?$CJ?$FLLjava?1lan@ 1000d6f4     java_md.obj
 0002:00002720       ??_C@_0L@BJEEEGHP@expandArgs@ 1000d720     java_md.obj
 0002:0000272c       ??_C@_06GLDDLHNF@malloc@   1000d72c     jli_util.obj
 0002:00002734       ??_C@_07EOOHGPEI@realloc@  1000d734     jli_util.obj
 0002:0000273c       ??_C@_06GFPDKFFG@strdup@   1000d73c     jli_util.obj
 0002:00002744       ??_C@_0BF@LACNODFI@META?9INF?1MANIFEST?4MF@ 1000d744     parse_manifest.obj
 0002:0000275c       ??_C@_05OJPKCACG@1?43?41@  1000d75c     parse_manifest.obj
 0002:00002764       ??_C@_02LIIHNNHG@?6?$AN@   1000d764     parse_manifest.obj
 0002:00002768       ??_C@_0BB@NKLIEOFJ@Manifest?9Version@ 1000d768     parse_manifest.obj
 0002:0000277c       ??_C@_0L@CIHLCGEL@Main?9Class@ 1000d77c     parse_manifest.obj
 0002:00002788       ??_C@_0M@DJAFHGJP@JRE?9Version@ 1000d788     parse_manifest.obj
 0002:00002794       ??_C@_0BD@ODACGPCD@Splashscreen?9Image@ 1000d794     parse_manifest.obj
 0002:000027a8       ??_C@_0BB@PKAPNNLJ@SplashLoadMemory@ 1000d7a8     splashscreen_stubs.obj
 0002:000027bc       ??_C@_0P@JIPKACHN@SplashLoadFile@ 1000d7bc     splashscreen_stubs.obj
 0002:000027cc       ??_C@_0L@JOBDBDOP@SplashInit@ 1000d7cc     splashscreen_stubs.obj
 0002:000027d8       ??_C@_0BF@GABHKIKD@SplashSetFileJarName@ 1000d7d8     splashscreen_stubs.obj
 0002:000027f0       ??_C@_0BF@LIMBEMBN@SplashSetScaleFactor@ 1000d7f0     splashscreen_stubs.obj
 0002:00002808       ??_C@_0BJ@FJIBEMML@SplashGetScaledImageName@ 1000d808     splashscreen_stubs.obj
 0002:00002824       ??_C@_0CD@ECEPLAJG@SplashGetScaledImgNameMaxPstfix@ 1000d824     splashscreen_stubs.obj
 0002:00002848       ??_C@_03NODMINOH@jar@      1000d848     wildcard.obj
 0002:0000284c       ??_C@_03NDMHEAJL@JAR@      1000d84c     wildcard.obj
 0002:00002850       ??_C@_0DH@KEOBCGCG@Expanded?5wildcards?3?6?5?5?5?5before?3@ 1000d850     wildcard.obj
 0002:00005108       ??_C@_0BA@MOKMMFOD@need?5dictionary@ 10010108     zutil.obj
 0002:00005118       ??_C@_0L@FNAOCBOG@stream?5end@ 10010118     zutil.obj
 0002:00005124       ??_C@_0L@KIJFAKBJ@file?5error@ 10010124     zutil.obj
 0002:00005130       ??_C@_0N@MKKNPMJD@stream?5error@ 10010130     zutil.obj
 0002:00005140       ??_C@_0L@HAHMBNLP@data?5error@ 10010140     zutil.obj
 0002:0000514c       ??_C@_0BE@OGGJBMCE@insufficient?5memory@ 1001014c     zutil.obj
 0002:00005160       ??_C@_0N@DFPGLBGC@buffer?5error@ 10010160     zutil.obj
 0002:00005170       ??_C@_0BF@CJFPCCEG@incompatible?5version@ 10010170     zutil.obj
 0002:00005188       _z_errmsg                  10010188     zutil.obj
 0002:000051b8       __pRawDllMain              100101b8     MSVCRT:dll_dllmain.obj
 0002:000051b8       __pDefaultRawDllMain       100101b8     MSVCRT:dll_dllmain.obj
 0002:00005230       __load_config_used         10010230     MSVCRT:loadcfg.obj
 0002:000052d0       ___safe_se_handler_table   100102d0     <linker-defined>
 0002:00005554       ___rtc_iaa                 10010554     MSVCRT:initsect.obj
 0002:00005558       ___rtc_izz                 10010558     MSVCRT:initsect.obj
 0002:0000555c       ___rtc_taa                 1001055c     MSVCRT:initsect.obj
 0002:00005560       ___rtc_tzz                 10010560     MSVCRT:initsect.obj
 0002:00005864       __IMPORT_DESCRIPTOR_COMCTL32 10010864     comctl32:COMCTL32.dll
 0002:00005878       __IMPORT_DESCRIPTOR_USER32 10010878     user32:USER32.dll
 0002:0000588c       __IMPORT_DESCRIPTOR_KERNEL32 1001088c     kernel32:KERNEL32.dll
 0002:000058a0       __IMPORT_DESCRIPTOR_VCRUNTIME140 100108a0     vcruntime:VCRUNTIME140.dll
 0002:000058b4       __IMPORT_DESCRIPTOR_api-ms-win-crt-runtime-l1-1-0 100108b4     ucrt:api-ms-win-crt-runtime-l1-1-0.dll
 0002:000058c8       __IMPORT_DESCRIPTOR_api-ms-win-crt-environment-l1-1-0 100108c8     ucrt:api-ms-win-crt-environment-l1-1-0.dll
 0002:000058dc       __IMPORT_DESCRIPTOR_api-ms-win-crt-stdio-l1-1-0 100108dc     ucrt:api-ms-win-crt-stdio-l1-1-0.dll
 0002:000058f0       __IMPORT_DESCRIPTOR_api-ms-win-crt-filesystem-l1-1-0 100108f0     ucrt:api-ms-win-crt-filesystem-l1-1-0.dll
 0002:00005904       __IMPORT_DESCRIPTOR_api-ms-win-crt-string-l1-1-0 10010904     ucrt:api-ms-win-crt-string-l1-1-0.dll
 0002:00005918       __IMPORT_DESCRIPTOR_api-ms-win-crt-heap-l1-1-0 10010918     ucrt:api-ms-win-crt-heap-l1-1-0.dll
 0002:0000592c       __IMPORT_DESCRIPTOR_api-ms-win-crt-convert-l1-1-0 1001092c     ucrt:api-ms-win-crt-convert-l1-1-0.dll
 0002:00005940       __NULL_IMPORT_DESCRIPTOR   10010940     comctl32:COMCTL32.dll
 0003:00000028       _awtPreloadD3D             10012028     java_md.obj
 0003:00000040       ___security_cookie_complement 10012040     MSVCRT:gs_cookie.obj
 0003:00000044       ___security_cookie         10012044     MSVCRT:gs_cookie.obj
 0003:00000048       __fltused                  10012048     MSVCRT:fltused.obj
 0003:00000050       ___scrt_native_dllmain_reason 10012050     MSVCRT:utility.obj
 0003:00000060       ___isa_enabled             10012060     MSVCRT:cpu_disp.obj
 0003:00000064       ___scrt_ucrt_dll_is_in_use 10012064     MSVCRT:ucrt_stubs.obj
 0003:000000d8       _awtPreloaded              100120d8     java_md.obj
 0003:00000588       ?__type_info_root_node@@3U__type_info_node@@A 10012588     MSVCRT:tncleanup.obj
 0003:00000590       ___scrt_current_native_startup_state 10012590     MSVCRT:utility.obj
 0003:00000594       ___scrt_native_startup_lock 10012594     MSVCRT:utility.obj
 0003:000005b4       ___scrt_debugger_hook_flag 100125b4     MSVCRT:utility_desktop.obj
 0003:000005b8       ___isa_available           100125b8     MSVCRT:cpu_disp.obj
 0003:000005bc       ___favor                   100125bc     MSVCRT:cpu_disp.obj
 0003:000005c0       ?_OptionsStorage@?1??__local_stdio_scanf_options@@9@9 100125c0     <common>
 0003:000005c8       ?_OptionsStorage@?1??__local_stdio_printf_options@@9@9 100125c8     <common>
 0003:000005d0       ___dyn_tls_init_callback   100125d0     <common>

 entry point at        0001:000093f2

 Static symbols

 0000:fffeb000       .debug$S                   10000000     ucrt:api-ms-win-crt-string-l1-1-0.dll
 0000:fffeb000       .debug$S                   10000000     user32:USER32.dll
 0000:fffeb000       .debug$S                   10000000     user32:USER32.dll
 0000:fffeb000       .debug$S                   10000000     kernel32:KERNEL32.dll
 0000:fffeb000       .debug$S                   10000000     kernel32:KERNEL32.dll
 0000:fffeb000       .debug$S                   10000000     kernel32:KERNEL32.dll
 0000:fffeb000       .debug$S                   10000000     kernel32:KERNEL32.dll
 0000:fffeb000       .debug$S                   10000000     kernel32:KERNEL32.dll
 0000:fffeb000       .debug$S                   10000000     kernel32:KERNEL32.dll
 0000:fffeb000       .debug$S                   10000000     kernel32:KERNEL32.dll
 0000:fffeb000       .debug$S                   10000000     kernel32:KERNEL32.dll
 0000:fffeb000       .debug$S                   10000000     kernel32:KERNEL32.dll
 0000:fffeb000       .debug$S                   10000000     kernel32:KERNEL32.dll
 0000:fffeb000       .debug$S                   10000000     kernel32:KERNEL32.dll
 0000:fffeb000       .debug$S                   10000000     kernel32:KERNEL32.dll
 0000:fffeb000       .debug$S                   10000000     kernel32:KERNEL32.dll
 0000:fffeb000       .debug$S                   10000000     kernel32:KERNEL32.dll
 0000:fffeb000       .debug$S                   10000000     kernel32:KERNEL32.dll
 0000:fffeb000       .debug$S                   10000000     kernel32:KERNEL32.dll
 0000:fffeb000       .debug$S                   10000000     kernel32:KERNEL32.dll
 0000:fffeb000       .debug$S                   10000000     kernel32:KERNEL32.dll
 0000:fffeb000       .debug$S                   10000000     kernel32:KERNEL32.dll
 0000:fffeb000       .debug$S                   10000000     kernel32:KERNEL32.dll
 0000:fffeb000       .debug$S                   10000000     kernel32:KERNEL32.dll
 0000:fffeb000       .debug$S                   10000000     jli.exp
 0000:fffeb000       .debug$S                   10000000     kernel32:KERNEL32.dll
 0000:fffeb000       .debug$S                   10000000     kernel32:KERNEL32.dll
 0000:fffeb000       .debug$S                   10000000     kernel32:KERNEL32.dll
 0000:fffeb000       .debug$S                   10000000     kernel32:KERNEL32.dll
 0000:fffeb000       .debug$S                   10000000     kernel32:KERNEL32.dll
 0000:fffeb000       .debug$S                   10000000     kernel32:KERNEL32.dll
 0000:fffeb000       .debug$S                   10000000     kernel32:KERNEL32.dll
 0000:fffeb000       .debug$S                   10000000     kernel32:KERNEL32.dll
 0000:fffeb000       .debug$S                   10000000     ucrt:api-ms-win-crt-stdio-l1-1-0.dll
 0000:fffeb000       .debug$S                   10000000     ucrt:api-ms-win-crt-stdio-l1-1-0.dll
 0000:fffeb000       .debug$S                   10000000     ucrt:api-ms-win-crt-string-l1-1-0.dll
 0000:fffeb000       .debug$S                   10000000     ucrt:api-ms-win-crt-string-l1-1-0.dll
 0000:fffeb000       .debug$S                   10000000     ucrt:api-ms-win-crt-runtime-l1-1-0.dll
 0000:fffeb000       .debug$S                   10000000     ucrt:api-ms-win-crt-runtime-l1-1-0.dll
 0000:fffeb000       .debug$S                   10000000     ucrt:api-ms-win-crt-runtime-l1-1-0.dll
 0000:fffeb000       .debug$S                   10000000     ucrt:api-ms-win-crt-runtime-l1-1-0.dll
 0000:fffeb000       .debug$S                   10000000     ucrt:api-ms-win-crt-runtime-l1-1-0.dll
 0000:fffeb000       .debug$S                   10000000     ucrt:api-ms-win-crt-runtime-l1-1-0.dll
 0000:fffeb000       .debug$S                   10000000     ucrt:api-ms-win-crt-runtime-l1-1-0.dll
 0000:fffeb000       .debug$S                   10000000     ucrt:api-ms-win-crt-runtime-l1-1-0.dll
 0000:fffeb000       .debug$S                   10000000     ucrt:api-ms-win-crt-runtime-l1-1-0.dll
 0000:fffeb000       .debug$S                   10000000     ucrt:api-ms-win-crt-runtime-l1-1-0.dll
 0000:fffeb000       .debug$S                   10000000     ucrt:api-ms-win-crt-runtime-l1-1-0.dll
 0000:fffeb000       .debug$S                   10000000     ucrt:api-ms-win-crt-runtime-l1-1-0.dll
 0000:fffeb000       .debug$S                   10000000     ucrt:api-ms-win-crt-stdio-l1-1-0.dll
 0000:fffeb000       .debug$S                   10000000     ucrt:api-ms-win-crt-string-l1-1-0.dll
 0000:fffeb000       .debug$S                   10000000     ucrt:api-ms-win-crt-heap-l1-1-0.dll
 0000:fffeb000       .debug$S                   10000000     ucrt:api-ms-win-crt-runtime-l1-1-0.dll
 0000:fffeb000       .debug$S                   10000000     ucrt:api-ms-win-crt-stdio-l1-1-0.dll
 0000:fffeb000       .debug$S                   10000000     ucrt:api-ms-win-crt-convert-l1-1-0.dll
 0000:fffeb000       .debug$S                   10000000     ucrt:api-ms-win-crt-filesystem-l1-1-0.dll
 0000:fffeb000       .debug$S                   10000000     ucrt:api-ms-win-crt-heap-l1-1-0.dll
 0000:fffeb000       .debug$S                   10000000     ucrt:api-ms-win-crt-heap-l1-1-0.dll
 0000:fffeb000       .debug$S                   10000000     ucrt:api-ms-win-crt-runtime-l1-1-0.dll
 0000:fffeb000       .debug$S                   10000000     ucrt:api-ms-win-crt-stdio-l1-1-0.dll
 0000:fffeb000       .debug$S                   10000000     ucrt:api-ms-win-crt-stdio-l1-1-0.dll
 0000:fffeb000       .debug$S                   10000000     ucrt:api-ms-win-crt-filesystem-l1-1-0.dll
 0000:fffeb000       .debug$S                   10000000     ucrt:api-ms-win-crt-string-l1-1-0.dll
 0000:fffeb000       .debug$S                   10000000     ucrt:api-ms-win-crt-runtime-l1-1-0.dll
 0000:fffeb000       .debug$S                   10000000     ucrt:api-ms-win-crt-string-l1-1-0.dll
 0000:fffeb000       .debug$S                   10000000     ucrt:api-ms-win-crt-string-l1-1-0.dll
 0000:fffeb000       .debug$S                   10000000     ucrt:api-ms-win-crt-runtime-l1-1-0.dll
 0000:fffeb000       .debug$S                   10000000     ucrt:api-ms-win-crt-runtime-l1-1-0.dll
 0000:fffeb000       .debug$S                   10000000     ucrt:api-ms-win-crt-string-l1-1-0.dll
 0000:fffeb000       .debug$S                   10000000     ucrt:api-ms-win-crt-string-l1-1-0.dll
 0000:fffeb000       .debug$S                   10000000     ucrt:api-ms-win-crt-string-l1-1-0.dll
 0000:fffeb000       .debug$S                   10000000     ucrt:api-ms-win-crt-string-l1-1-0.dll
 0000:fffeb000       .debug$S                   10000000     ucrt:api-ms-win-crt-environment-l1-1-0.dll
 0000:fffeb000       .debug$S                   10000000     ucrt:api-ms-win-crt-heap-l1-1-0.dll
 0000:fffeb000       .debug$S                   10000000     ucrt:api-ms-win-crt-stdio-l1-1-0.dll
 0000:fffeb000       .debug$S                   10000000     ucrt:api-ms-win-crt-stdio-l1-1-0.dll
 0000:fffeb000       .debug$S                   10000000     ucrt:api-ms-win-crt-stdio-l1-1-0.dll
 0000:fffeb000       .debug$S                   10000000     ucrt:api-ms-win-crt-stdio-l1-1-0.dll
 0000:fffeb000       .debug$S                   10000000     ucrt:api-ms-win-crt-stdio-l1-1-0.dll
 0000:fffeb000       .debug$S                   10000000     comctl32:COMCTL32.dll
 0000:fffeb000       .debug$S                   10000000     ucrt:api-ms-win-crt-string-l1-1-0.dll
 0000:fffeb000       .debug$S                   10000000     ucrt:api-ms-win-crt-string-l1-1-0.dll
 0000:fffeb000       .debug$S                   10000000     ucrt:api-ms-win-crt-filesystem-l1-1-0.dll
 0000:fffeb000       .debug$S                   10000000     ucrt:api-ms-win-crt-stdio-l1-1-0.dll
 0000:fffeb000       .debug$S                   10000000     ucrt:api-ms-win-crt-stdio-l1-1-0.dll
 0000:fffeb000       .debug$S                   10000000     ucrt:api-ms-win-crt-stdio-l1-1-0.dll
 0000:fffeb000       .debug$S                   10000000     ucrt:api-ms-win-crt-stdio-l1-1-0.dll
 0000:fffeb000       .debug$S                   10000000     ucrt:api-ms-win-crt-stdio-l1-1-0.dll
 0000:fffeb000       .debug$S                   10000000     ucrt:api-ms-win-crt-environment-l1-1-0.dll
 0000:fffeb000       .debug$S                   10000000     ucrt:api-ms-win-crt-runtime-l1-1-0.dll
 0000:fffeb000       .debug$S                   10000000     kernel32:KERNEL32.dll
 0000:fffeb000       .debug$S                   10000000     vcruntime:VCRUNTIME140.dll
 0000:fffeb000       .debug$S                   10000000     vcruntime:VCRUNTIME140.dll
 0000:fffeb000       .debug$S                   10000000     vcruntime:VCRUNTIME140.dll
 0000:fffeb000       .debug$S                   10000000     vcruntime:VCRUNTIME140.dll
 0000:fffeb000       .debug$S                   10000000     vcruntime:VCRUNTIME140.dll
 0000:fffeb000       .debug$S                   10000000     vcruntime:VCRUNTIME140.dll
 0000:fffeb000       .debug$S                   10000000     vcruntime:VCRUNTIME140.dll
 0000:fffeb000       .debug$S                   10000000     vcruntime:VCRUNTIME140.dll
 0000:fffeb000       .debug$S                   10000000     kernel32:KERNEL32.dll
 0001:00000135       _checkArg                  10001135 f   args.obj
 0001:000001dd       _expand                    100011dd f   args.obj
 0001:00000387       _expandArgFile             10001387 f   args.obj
 0001:00000519       _nextToken                 10001519 f   args.obj
 0001:00000775       _readArgFile               10001775 f   args.obj
 0001:000009fe       _copyCh                    100019fe f   cmdtoargs.obj
 0001:00000a1c       _next_arg                  10001a1c f   cmdtoargs.obj
 0001:00002643       $LN767                     10003643     inflate.obj
 0001:000028b9       _inflateStateCheck         100038b9 f   inflate.obj
 0001:000028ec       _updatewindow              100038ec f   inflate.obj
 0001:00002ddb       _AddApplicationOptions     10003ddb f   java.obj
 0001:00002f66       _AddLongFormOption         10003f66 f   java.obj
 0001:00003417       _DescribeModule            10004417 f   java.obj
 0001:00003475       _DumpState                 10004475 f   java.obj
 0001:00003522       _GetApplicationClass       10004522 f   java.obj
 0001:000035ae       _GetOpt                    100045ae f   java.obj
 0001:000036d6       _InitializeJVM             100046d6 f   java.obj
 0001:0000379e       _IsClassPathOption         1000479e f   java.obj
 0001:000037e0       _IsLauncherMainOption      100047e0 f   java.obj
 0001:0000380e       _IsLauncherOption          1000480e f   java.obj
 0001:00003864       _IsLongFormModuleOption    10004864 f   java.obj
 0001:000038e8       _IsModuleOption            100048e8 f   java.obj
 0001:00003992       _IsOptionWithArgument      10004992 f   java.obj
 0001:00004182       _KnownVMIndex              10005182 f   java.obj
 0001:000041d4       _ListModules               100051d4 f   java.obj
 0001:0000421d       _LoadMainClass             1000521d f   java.obj
 0001:000042f5       _NewPlatformString         100052f5 f   java.obj
 0001:0000443d       _ParseArguments            1000543d f   java.obj
 0001:00004d6d       _PrintJavaVersion          10005d6d f   java.obj
 0001:00004dd2       _PrintUsage                10005dd2 f   java.obj
 0001:00005366       _SelectVersion             10006366 f   java.obj
 0001:000055bb       _SetClassPath              100065bb f   java.obj
 0001:000056c3       _SetJvmEnvironment         100066c3 f   java.obj
 0001:000057f0       _ShowResolvedModules       100067f0 f   java.obj
 0001:00005839       _ShowSettings              10006839 f   java.obj
 0001:000059f4       _TranslateApplicationArgs  100069f4 f   java.obj
 0001:00005bdb       _checkMode                 10006bdb f   java.obj
 0001:00005bff       _expandWildcardOnLongOpt   10006bff f   java.obj
 0001:00005ca1       _parse_size                10006ca1 f   java.obj
 0001:000065e4       _GetJREPath                100075e4 f   java_md.obj
 0001:0000671a       _GetJVMPath                1000771a f   java_md.obj
 0001:00006c12       _LoadMSVCRT                10007c12 f   java_md.obj
 0001:00006e2a       _ThreadJavaMain@4          10007e2a f   java_md.obj
 0001:00007511       _find_file                 10008511 f   parse_manifest.obj
 0001:00007892       _find_positions            10008892 f   parse_manifest.obj
 0001:00007a4a       _find_positions64          10008a4a f   parse_manifest.obj
 0001:00007e1f       _inflate_file              10008e1f f   parse_manifest.obj
 0001:00007f5d       _is_valid_end_header       10008f5d f   parse_manifest.obj
 0001:00008099       _is_zip64_endhdr           10009099 f   parse_manifest.obj
 0001:000082d0       _parse_nv_pair             100092d0 f   parse_manifest.obj
 0001:00008399       _readAt                    10009399 f   parse_manifest.obj
 0001:000084df       _FileList_expandWildcards  100094df f   wildcard.obj
 0001:00008666       _wildcardFileList          10009666 f   wildcard.obj
 0001:00008cb7       _crc_word                  10009cb7 f   zcrc32.obj
 0001:00008d00       $$000000                   10009d00     MSVCRT:chkstk.obj
 0001:00008f30       $$000000                   10009f30     MSVCRT:lldiv.obj
 0001:00008fe0       $$000000                   10009fe0     MSVCRT:llmul.obj
 0001:00009020       $$000000                   1000a020     MSVCRT:llrem.obj
 0001:000090d2       ?dllmain_crt_dispatch@@YGHQAUHINSTANCE__@@KQAX@Z 1000a0d2 f   MSVCRT:dll_dllmain.obj
 0001:00009125       ?dllmain_crt_process_attach@@YAHQAUHINSTANCE__@@QAX@Z 1000a125 f   MSVCRT:dll_dllmain.obj
 0001:0000922f       ?dllmain_crt_process_detach@@YAH_N@Z 1000a22f f   MSVCRT:dll_dllmain.obj
 0001:000092c1       ?dllmain_dispatch@@YAHQAUHINSTANCE__@@KQAX@Z 1000a2c1 f   MSVCRT:dll_dllmain.obj
 0001:000093c7       ?dllmain_raw@@YGHQAUHINSTANCE__@@KQAX@Z 1000a3c7 f   MSVCRT:dll_dllmain.obj
 0001:00009415       ___get_entropy             1000a415 f   MSVCRT:gs_support.obj
 0001:00009504       ?find_pe_section@@YAPAU_IMAGE_SECTION_HEADER@@QAEI@Z 1000a504 f   MSVCRT:utility.obj
 0001:00009980       $$000000                   1000a980     MSVCRT:sehprolg4.obj
 0002:00000508       ?lenfix@?1??fixedtables@@9@9 1000b508     inflate.obj
 0002:00000d08       ?distfix@?1??fixedtables@@9@9 1000bd08     inflate.obj
 0002:00000d88       ?order@?1??inflate@@9@9    1000bd88     inflate.obj
 0002:00000f78       ?lbase@?1??inflate_table@@9@9 1000bf78     inftrees.obj
 0002:00000fb8       ?lext@?1??inflate_table@@9@9 1000bfb8     inftrees.obj
 0002:00000ff8       ?dbase@?1??inflate_table@@9@9 1000bff8     inftrees.obj
 0002:00001038       ?dext@?1??inflate_table@@9@9 1000c038     inftrees.obj
 0002:00001084       ?format@?1??SetClassPath@@9@9 1000c084     java.obj
 0002:0000109c       ?format@?1??AddLongFormOption@@9@9 1000c09c     java.obj
 0002:000010a4       ?format@?1??SetMainModule@@9@9 1000c0a4     java.obj
 0002:00002888       _crc_table                 1000d888     zcrc32.obj
 0002:00002c88       _crc_big_table             1000dc88     zcrc32.obj
 0002:00003088       _crc_braid_table           1000e088     zcrc32.obj
 0002:00004088       _crc_braid_big_table       1000f088     zcrc32.obj
 0002:00005088       _x2n_table                 10010088     zcrc32.obj
 0002:000051b0       _GS_ExceptionPointers      100101b0     MSVCRT:gs_report.obj
 0002:00005568       __sehtable$?dllmain_crt_process_attach@@YAHQAUHINSTANCE__@@QAX@Z 10010568     MSVCRT:dll_dllmain.obj
 0002:00005588       __sehtable$?dllmain_crt_process_detach@@YAH_N@Z 10010588     MSVCRT:dll_dllmain.obj
 0002:000055a8       __sehtable$?dllmain_dispatch@@YAHQAUHINSTANCE__@@KQAX@Z 100105a8     MSVCRT:dll_dllmain.obj
 0002:000055c8       __sehtable$___scrt_is_nonwritable_in_current_image 100105c8     MSVCRT:utility.obj
 0002:000055f0       .edata                     100105f0     jli.exp
 0002:00005618       rgpv                       10010618     jli.exp
 0002:00005664       rgszName                   10010664     jli.exp
 0002:000056b0       rgwOrd                     100106b0     jli.exp
 0002:000056d6       szName                     100106d6     jli.exp
 0002:000056de       $N00001                    100106de     jli.exp
 0002:000056f7       $N00002                    100106f7     jli.exp
 0002:00005708       $N00003                    10010708     jli.exp
 0002:0000571e       $N00004                    1001071e     jli.exp
 0002:00005730       $N00005                    10010730     jli.exp
 0002:00005742       $N00006                    10010742     jli.exp
 0002:0000575b       $N00007                    1001075b     jli.exp
 0002:0000576a       $N00008                    1001076a     jli.exp
 0002:0000577a       $N00009                    1001077a     jli.exp
 0002:0000578a       $N00010                    1001078a     jli.exp
 0002:000057a2       $N00011                    100107a2     jli.exp
 0002:000057b2       $N00012                    100107b2     jli.exp
 0002:000057c1       $N00013                    100107c1     jli.exp
 0002:000057d6       $N00014                    100107d6     jli.exp
 0002:000057ed       $N00015                    100107ed     jli.exp
 0002:00005807       $N00016                    10010807     jli.exp
 0002:00005829       $N00017                    10010829     jli.exp
 0002:0000583b       $N00018                    1001083b     jli.exp
 0002:00005853       $N00019                    10010853     jli.exp
 0002:00005b08       .idata$6                   10010b08     comctl32:COMCTL32.dll
 0002:00005b32       .idata$6                   10010b32     user32:USER32.dll
 0002:00005d82       .idata$6                   10010d82     kernel32:KERNEL32.dll
 0002:00005e06       .idata$6                   10010e06     vcruntime:VCRUNTIME140.dll
 0002:000060c8       .idata$6                   100110c8     ucrt:api-ms-win-crt-runtime-l1-1-0.dll
 0002:000060ea       .idata$6                   100110ea     ucrt:api-ms-win-crt-environment-l1-1-0.dll
 0002:00006110       .idata$6                   10011110     ucrt:api-ms-win-crt-stdio-l1-1-0.dll
 0002:00006130       .idata$6                   10011130     ucrt:api-ms-win-crt-filesystem-l1-1-0.dll
 0002:00006156       .idata$6                   10011156     ucrt:api-ms-win-crt-string-l1-1-0.dll
 0002:00006178       .idata$6                   10011178     ucrt:api-ms-win-crt-heap-l1-1-0.dll
 0002:00006198       .idata$6                   10011198     ucrt:api-ms-win-crt-convert-l1-1-0.dll
 0003:00000000       _firstAppArgIndex          10012000     args.obj
 0003:00000004       _argsCount                 10012004     args.obj
 0003:00000008       _launchModeNames           10012008     java.obj
 0003:0000001c       _printTo                   1001201c     java.obj
 0003:00000020       ?NMT_Env_Name@?1??SetJvmEnvironment@@9@9 10012020     java.obj
 0003:00000024       ?whiteSpace@?1??ReadKnownVMs@@9@9 10012024     java.obj
 0003:0000002c       _SPLASHSCREEN_SO           1001202c     java_md.obj
 0003:00000030       _manifest_name             10012030     parse_manifest.obj
 0003:00000068       _expectingNoDashArg        10012068     args.obj
 0003:00000069       _stopExpansion             10012069     args.obj
 0003:0000006a       _relaunch                  1001206a     args.obj
 0003:0000006c       _stdargs                   1001206c     cmdtoargs.obj
 0003:00000070       _stdargc                   10012070     cmdtoargs.obj
 0003:00000078       _printVersion              10012078     java.obj
 0003:00000079       _showVersion               10012079     java.obj
 0003:0000007a       _printUsage                1001207a     java.obj
 0003:0000007b       _printXUsage               1001207b     java.obj
 0003:0000007c       _dryRun                    1001207c     java.obj
 0003:0000007d       _showResolvedModules       1001207d     java.obj
 0003:0000007e       _listModules               1001207e     java.obj
 0003:0000007f       _validateModules           1001207f     java.obj
 0003:00000080       _showSettings              10012080     java.obj
 0003:00000084       _describeModule            10012084     java.obj
 0003:00000088       __program_name             10012088     java.obj
 0003:0000008c       __launcher_name            1001208c     java.obj
 0003:00000090       __is_java_args             10012090     java.obj
 0003:00000091       __have_classpath           10012091     java.obj
 0003:00000092       __wc_enabled               10012092     java.obj
 0003:00000094       __fVersion                 10012094     java.obj
 0003:00000098       _splash_file_entry         10012098     java.obj
 0003:0000009c       _splash_jar_entry          1001209c     java.obj
 0003:000000a0       _options                   100120a0     java.obj
 0003:000000a4       _numOptions                100120a4     java.obj
 0003:000000a8       _maxOptions                100120a8     java.obj
 0003:000000ac       _knownVMs                  100120ac     java.obj
 0003:000000b0       _knownVMsCount             100120b0     java.obj
 0003:000000b4       _knownVMsLimit             100120b4     java.obj
 0003:000000b8       _threadStackSize           100120b8     java.obj
 0003:000000c0       _maxHeapSize               100120c0     java.obj
 0003:000000c8       _initialHeapSize           100120c8     java.obj
 0003:000000d0       _helperClass               100120d0     java.obj
 0003:000000d4       _makePlatformStringMID     100120d4     java.obj
 0003:000000dc       __isjavaw                  100120dc     java_md.obj
 0003:000000dd       _counterAvailable          100120dd     java_md.obj
 0003:000000de       _counterInitialized        100120de     java_md.obj
 0003:000000e0       ?loaded@?1??LoadMSVCRT@@9@9 100120e0     java_md.obj
 0003:000000e4       _hSplashLib                100120e4     java_md.obj
 0003:000000e8       _counterFrequency          100120e8     java_md.obj
 0003:000000f0       _findBootClass             100120f0     java_md.obj
 0003:000000f4       _fnPreloadStop             100120f4     java_md.obj
 0003:000000f8       _hPreloadAwt               100120f8     java_md.obj
 0003:000000fc       __launcher_debug           100120fc     jli_util.obj
 0003:00000100       _manifest                  10012100     parse_manifest.obj
 0003:00000104       ?proc@?1??DoSplashLoadMemory@@9@9 10012104     splashscreen_stubs.obj
 0003:00000108       ?proc@?1??DoSplashLoadFile@@9@9 10012108     splashscreen_stubs.obj
 0003:0000010c       ?proc@?1??DoSplashInit@@9@9 1001210c     splashscreen_stubs.obj
 0003:00000110       ?proc@?1??DoSplashClose@@9@9 10012110     splashscreen_stubs.obj
 0003:00000114       ?proc@?1??DoSplashSetFileJarName@@9@9 10012114     splashscreen_stubs.obj
 0003:00000118       ?proc@?1??DoSplashSetScaleFactor@@9@9 10012118     splashscreen_stubs.obj
 0003:0000011c       ?proc@?1??DoSplashGetScaledImageName@@9@9 1001211c     splashscreen_stubs.obj
 0003:00000120       ?proc@?1??DoSplashGetScaledImgNameMaxPstfixLen@@9@9 10012120     splashscreen_stubs.obj
 0003:00000128       _find_data                 10012128     wildcard.obj
 0003:00000268       _GS_ExceptionRecord        10012268     MSVCRT:gs_report.obj
 0003:000002b8       _GS_ContextRecord          100122b8     MSVCRT:gs_report.obj
 0003:00000584       ?__proc_attached@@3HA      10012584     MSVCRT:dll_dllmain.obj
 0003:00000598       ?is_initialized_as_dll@@3_NA 10012598     MSVCRT:utility.obj
 0003:00000599       ?module_local_atexit_table_initialized@@3_NA 10012599     MSVCRT:utility.obj
 0003:0000059c       ?module_local_atexit_table@@3U_onexit_table_t@@A 1001259c     MSVCRT:utility.obj
 0003:000005a8       ?module_local_at_quick_exit_table@@3U_onexit_table_t@@A 100125a8     MSVCRT:utility.obj
 0004:00000060       $R000000                   10013060     jli.dll.res
